:10000000004000203D6200007D6200007F62000031
:1000100000000000000000000000000000000000E0
:1000200000000000000000000000000081620000ED
:1000300000000000000000008362000085620000F4
:1000400087620000812D0000716A00008762000055
:1000500087620000000000008762000087620000E5
:1000600087620000B56400008762000087620000BC
:1000700087620000876200008762000087620000DC
:1000800087620000156B0000876200008762000035
:1000900087620000876200008762000087620000BC
:1000A000876200008762000000000000000000007E
:1000B0000000000000000000000000000000000040
:1000C000054B0648033310B51B1A062B03D9044B06
:1000D000002B00D0984710BD4002002040020020B5
:1000E000000000000648074910B5091A8910CB0F17
:1000F0005918491003D0044B002B00D0984710BD6D
:1001000040020020400200200000000010B5074C13
:100110002378002B09D1FFF7D3FF054B002B02D02A
:10012000044800E000BF0123237010BD40020020FE
:100130000000000010AE0000094B10B5002B03D0EA
:100140000849094800E000BF08480368002B02D1B5
:10015000FFF7C8FF10BD064B002BF9D09847F7E713
:10016000000000004402002010AE00003C0200200D
:1001700000000000164B002B00D1144B9D4640227E
:1001800092029A1A924600218B460F461348144A4F
:10019000121A08F0C8FB0F4B002B00D098470E4BEB
:1001A000002B00D098470020002104000D000D48CE
:1001B000002802D00C4800E000BF08F071FB2000CE
:1001C000290006F06DFC08F045FBC0460000080061
:1001D000004000200000000000000000400200205D
:1001E000F024002000000000000000000123034074
:1001F0000200181E04D1042A03D91068000900E087
:100200000020704710B50400FFF7F0FF0300002046
:1002100083420BD0013B9B00181DE2181279002A83
:1002200003D001338342F8D100E0180010BD012251
:10023000016810B5114201D0002903DA102000F046
:10024000AFF903E04910062001F0E8FE10BD016897
:1002500010B5CB0701D5002903DA102000F0A0F972
:1002600006E04910033189100022052001F0D6FE76
:1002700010BD70B50568AB0728D1042D26D90F2312
:100280002A6846681340062B09D12800FFF7AEFF05
:10029000012383421DDC9A00AE500133F9E7052BA0
:1002A00014D1F30703D4132000F07AF912E076108A
:1002B000FF2EF8D82800FFF799FF2C1D230080009F
:1002C0002018984205D91E700133FAE70B2000F080
:1002D00067F9002070BD70B50468E30701D41120F0
:1002E0002DE04568AB0729D1042D27D90F262B68AF
:1002F00064101E40062E0BD1002C04DD2800FFF7F1
:1003000075FF844201DD122019E0A400605918E055
:10031000331F012B12D82800FFF768FF8000042E3E
:1003200002D12800FFF76EFF002CECDDA042EADBD3
:1003300001232C19E0784000184302E00B2000F064
:100340002FF970BDF8B5012304681C4201D11120BA
:100350002FE00325466835402AD1042E28D90F23E3
:100360003268641087681340062B0BD1002C04DD23
:100370003000FFF73BFF844201DD122019E0A400AA
:10038000A75113E0052B13D1002CF6DD3000FFF749
:100390002DFF80008442F0DC01231F4201D1132095
:1003A00007E07F10FF2FFAD83419E770280002E029
:1003B0000B2000F0F5F8F8BD006810B5830717D1E1
:1003C000042815D90F2302681340062B02D1FFF72A
:1003D0000DFF0BE0052B05D1FFF708FFC00001233F
:1003E000184308E0042B03D1FFF70CFF4000F6E7A9
:1003F0000B2000F0D5F810BD10B5032400680440B0
:1004000006D1042804D90F2302681340042B01D01D
:100410000E2011E001F03EFE0378233B5942594182
:1004200010224018210008F057FF80239B05C218B6
:10043000054B9A4203D9142000F0B2F802E00123E0
:100440004000184310BDC046FFFFFF3F012303409B
:100450000200181E01D0501002E00D22014B1A704C
:100460007047C0465C020020012303400200181EB2
:1004700004D1042A03D91068000900E00020704765
:1004800070B50D000400FFF7EFFF86002800FFF7AE
:10049000EBFF830000209E420ED1231D9E190435E0
:1004A0001A009E4207D929781278013301358A4211
:1004B000F6D0002000E0012070BD0000F0B585B04E
:1004C0000393019002912D4E2D4B002A02D002225F
:1004D0003270013A00251A601B68F554019B9D4259
:1004E0004ADA029AAB00D058254B1C68C8239B00FF
:1004F00037191C1B0123184202D04310214A1FE068
:10050000214A002802D0042805D1204A21003800C1
:1005100008F0D0FD18E0042810D90F23026813401A
:10052000042B04D101F0B6FD194A030008E0062BA4
:1005300005D1FFF799FF174A030001E00123164A8E
:100540002100380008F0B6FD300008F019FE039BCA
:100550000B4A002B01D110600CE0019B013B9D4236
:10056000F9DA0E4B9842F6DC431C13602022325419
:100570000022F2540135B1E705B0F0BD6802002059
:1005800064020020A5A0000078A000007EA000006A
:10059000D6A3000083A0000094A000001F03000069
:1005A000014B1870002070475C02002070B503F00A
:1005B0003FFA094C0100251D1F22280008F0E7FD25
:1005C000280008F0DDFD04230430800800011843F2
:1005D0002060200070BDC04688050020C368F0B5CB
:1005E0009D00836889B05D19030018330693036981
:1005F00003909F00069BDF1943699E000193069BB1
:100600009E19D24B1B78002B0FD17F222B68D0492B
:100610001C1213409B005B5801960435029235E092
:10062000CA4B1B78002B29D0019E039BC74C9B68AB
:1006300021780193EA1A039B92109B7812021A43C5
:10064000039B587802F080FF0023039A23701370F5
:1006500001960497039B069A9B68ED1A0293039BED
:10066000AD10DD60049B9F1A039BBF101F61019BAF
:100670009B1A039A9B10536101F01EFC2B68029A8F
:100680001C121340B24A9B009B5804359F46039BA3
:10069000587802F051FF0023039A1370D9E7069BA4
:1006A0003A1DD11AA94BDB2903DD1A22019E1A70CB
:1006B000BBE71B783C60002B02D0019E1700B4E71B
:1006C0002B6802991C120B40A1499B005B58170034
:1006D0000435DBE7069B3A1DD11A9C4BDB2903DD71
:1006E0001A22019E1A70A0E728681B78291D38601D
:1006F000002B03D0019E17000D0096E76B6802994E
:100700001C120B4092499B005B5817000835BDE74F
:10071000069B3A1DD11A8D4BDB2903DD1A22019E5F
:100720001A7082E7A4001B782C193C60002B02D0C1
:10073000019E170079E72B6802991C120B4084492F
:100740009B005B5817000435A0E7069B3A1DD11AA1
:100750007E4BDB2903DD1A22019E1A7065E77D4876
:10076000A40021581B783960002B02D0019E17008D
:100770005BE72B6802991C120B4075499B005B5884
:100780001700043582E7043F724B3A68A400E25038
:100790006E4B1B78002B01D0019E46E72B68029A16
:1007A0001C1213406A4A9B009B5804356EE7694B44
:1007B000A600F058FFF74AFE043F04003868FFF730
:1007C00045FE24180120634B64000443F4505F4B42
:1007D0001B78002B01D0019E27E72B68029A1C1280
:1007E00013405B4A9B009B5804354FE7069B3A1D1C
:1007F000D11A564BDB2903DD1A22019E1A7014E729
:100800000198069C0121A04202D901000C39096817
:100810001B783960002B02D0019E170005E72B687A
:1008200002991C120B404A499B005B581700043583
:100830002CE7069B3A1DD11A444BDB2903DD1A2213
:10084000019E1A70F1E60199069881420AD90B00BF
:100850000C3B1B6840495B106418E41A019BA40020
:10086000E35802E01821197000233B60374B1B78D6
:10087000002B02D0019E1700D7E62B6802991C12AC
:100880000B4033499B005B5817000435FEE6019B83
:10089000069A93420BD90C3B19682F4B043FE3187F
:1008A0004910591A3A68019B8900CA5002E018227F
:1008B000264B1A70254B1B78002B01D0019EB4E605
:1008C0002B68029A1C121340214A9B009B58043546
:1008D000DCE6019B069A93421CD9019E1E4B0C3EFE
:1008E000E4183368019A5B10E31A9B009858FFF7ED
:1008F000ADFD043F04903868FFF7A8FD3168049B04
:100900004910611A012418184000019B89002043F6
:10091000C85002E018220D4B1A700C4B1B78002BAC
:1009200001D0019E81E62B68029A1C121340084AEE
:100930009B009B580435A9E6069B3A1DD11A034B30
:10094000DB290BDD1A22019E1A706EE65C02002084
:10095000789E000058230020FDFFFF3F0199A4006E
:1009600061581B783960002B02D0019E17005CE6AD
:100970002B6802991C120B40D0499B005B58170052
:10098000043583E6043F019B3A68A400E250CC4B57
:100990001B78002B01D0019E47E62B68029A1C129F
:1009A0001340C64A9B009B5804356FE6019BA40088
:1009B0001C192368043F38685E10FFF747FD36189E
:1009C0000120BF4B76001B7806432660002B01D028
:1009D000019E2AE62B68029A1C121340B74A9B001C
:1009E0009B58043552E6069BA4003F1BB44CBB4207
:1009F0000DD82378002B01D0019E16E62B68029AB1
:100A00001C121340AD4A9B009B5804353EE6AD488E
:100A100001F0B6FA2378002B01D0019E05E62B6881
:100A2000029A1C121340A54A9B009B5804352DE6E0
:100A3000A300ED18002C00DA0BE6A14B1B78002B6D
:100A400001D0019EF1E52B68029A1C1213409B4ACB
:100A50009B009B58043519E63B1F04931B680793C2
:100A6000042B04D1A300ED18002C00DAF2E5944B1E
:100A70001B78002B02D0019E049FD6E52B68029ABA
:100A80001C1213408D4A9B009B58049F0435FDE5C2
:100A90003B1F04931B68042B06D0A200AD18002C4A
:100AA00002DA002B00D1D5E5854B1B78002B02D054
:100AB000019E049FB9E52B68029A1C1213407F4ADD
:100AC0009B009B58049F0435E0E53A1F13685B10B8
:100AD000013B002B07DD01215B00A4000B430497C1
:100AE0002D191360B6E5764B17001B78002B01D04B
:100AF000019E9AE52B68029A1C1213406F4A9B00D4
:100B00009B580435C2E53A00069B0C32D31ADB2B06
:100B100004DD1A226A4B019E1A7086E5FF236100EC
:100B20005B000B4001210B433B60039B06989B68D5
:100B300024120493ED1A039BAD109B782D021D43E4
:100B4000019B8D401B1A9B108B400B43BB60039B8A
:100B50000D437D609C70E4B25B4BE4000399E35865
:100B600016008B6056490978002903D008331D0010
:100B700017005AE51D0002999B680C351C120B40AA
:100B80004E499B005B58019217007FE53B1F1E6892
:100B9000069A019B93422AD104970A20F30716D4A0
:100BA000B3070DD1042E0BD90F2332681340042B49
:100BB00006D1300001F06EFA08F0E2FA063006E0E5
:100BC0000720042E03D0002E01D080208000643046
:100BD00002F062FA002801D1043D3BE5039B31009D
:100BE000587802F0C3FC0023039A137032E5019B8E
:100BF000019A0C3B1B6803995B109B005B421F0032
:100C0000D3180C3B1E601300083B1B68083FD71924
:100C10005A108A70D2B22C49D2005B0055589B0AF8
:100C2000039A9B009560ED18019B043B1E68069B90
:100C30007610B6009E19224B1B78002B00D0F4E4EE
:100C40002B68029A1C1213401C4A9B009B58019669
:100C500004351BE53B1F1868FFF7F8FBA4000600EE
:100C60003F1B1E2834DC00280EDC154B1B78002BA4
:100C700001D0019ED9E42B68029A1C1213400F4A3E
:100C80009B009B58043501E502F0B8FE033E361880
:100C900002F0B4FE0D4B801B9842F9D8084B1B782C
:100CA000002B01D0019EC0E42B68029A1C12134055
:100CB000024A9B009B580435E8E4C046789E000039
:100CC0005C020020A8A00000601B00209F8601009D
:100CD0000123039A137002F091FE039B0A388619D0
:100CE0005E60B6E43B1F1868FFF7B0FBA4000490F9
:100CF0003F1B00280EDCCF4B1B78002B01D0019E40
:100D000093E42B68029A1C121340CB4A9B009B5819
:100D10000435BBE4C94B049A019E9A4203DD1D22AF
:100D2000C44B1A7081E40123039A137002F066FE2B
:100D3000FA23049A9B005343039A0A3B1B185360FF
:100D400087E4A300FF1A002320001A003900FFF7F0
:100D5000B5FBBB4EBB4C3168200002F053FB316841
:100D6000200002F00AFCB34B1B78002B01D0019E3F
:100D70005BE42B68029A1C121340AF4A9B009B58FD
:100D8000043583E4AB4BA4001B783F1B002B01D040
:100D9000019E4AE42B68029A1C121340A64A9B004B
:100DA0009B58043572E402F0BDF901F085F83B1F51
:100DB0001868002823D1083B1868C30701D54010E4
:100DC00016E083070FD104280DD90F2302681340C2
:100DD000062B02D1FFF748FB0AE0052B03D1FFF7F2
:100DE00043FB800004E01922924B019E1A701CE420
:100DF0003A0001214300083A0B43136001E0401020
:100E00000138002832DD012243001343391F0B60F3
:100E10003B00083B1B681341181A3B000C3B1B6846
:100E2000134203D08018A400904015E0990717D111
:100E3000042B15D90F211E683140062906D1013037
:100E40008000C358019AA400A35010E0052907D1DF
:100E500018180079A4004000019B1043E05006E000
:100E60001922744B019E1A70FFF7DFFB0435714B9A
:100E70001B78002B02D0019EFFF7D7FB2B68029A4C
:100E80001C1213406C4A9B009B580435FFF7FEFB75
:100E9000A300069AFB189B1ADB2B01DC012205E05C
:100EA0001A22644B019E1A70FFF7BFFB631E002CD1
:100EB00003DD3A601C000437F8E75E4B1B78002B1B
:100EC00002D0019EFFF7B1FB2B68029A1C1213405F
:100ED000594A9B009B580435FFF7D8FBA3009C465A
:100EE000F81A002C04DC1C22524B00261A7015E064
:100EF000002103685B1001268A008258164003D146
:100F00000D224C4B1A7009E05210934200DD130081
:100F100001318C42EFDC01265B001E436346FF1A61
:100F2000444B06601B780437002B02D0019EFFF76C
:100F30007CFB2B68029A1C1213403F4A9B009B5873
:100F40000435FFF7A3FBA3009C46F81A002C04DC31
:100F50001C22384B00261A7015E0002103685B1034
:100F600001268A008258164003D10D22314B1A7097
:100F700009E05210934200DA130001318C42EFDC99
:100F800001265B001E436346FF1A2A4B06601B784E
:100F90000437002B02D0019EFFF747FB2B68029A13
:100FA0001C121340244A9B009B580435FFF76EFB2C
:100FB0003B00083B1868FFF749FA3B1F049018688C
:100FC000FFF744FA049AA600BC1B0023824200DA11
:100FD00004332360174BBF1B1B780437002B02D050
:100FE000019EFFF722FB2B68029A1C121340124A43
:100FF0009B009B580435FFF749FBA300FE1A04939E
:101000003B00083B1868FFF721FA3B1F04001868F3
:10101000FFF71CFAE20FC317A04253419B00336055
:10102000049BFF1A034B04371B78002B0CD0019E46
:10103000FFF7FBFA5C020020789E000080EE36008D
:1010400064020020680200202B68029A1C121340E0
:10105000DB4A9B009B580435FFF718FB3B00083B1D
:1010600018683B1F1968A300884202D1FB1A0422AA
:1010700022E004281ED90122104201D0114219D1C8
:101080000326304215D10F2302681A40042A10D1DA
:1010900031420ED104290CD90A681340042B08D11F
:1010A000FFF7EEF9431E9841A600BE1B800030609A
:1010B00003E0A3000022FB1A1A60C24BA4001B78B5
:1010C0003F1B0437002B02D0019EFFF7AEFA2B68BE
:1010D000029A1C121340BA4A9B009B580435FFF732
:1010E000D5FA3B00083B18683B1F1968A3008842EB
:1010F00002D1FB1A002226E0042822D90122104244
:1011000004D0114202D0FB1A03321CE00326304205
:1011100016D10F2302681A40042A11D131420FD18F
:1011200004290DD90A681340042B09D1FFF7A8F947
:10113000030058425841A600BE1B8000306003E007
:10114000A3000422FB1A1A609E4BA4001B783F1BCD
:101150000437002B02D0019EFFF767FA2B68029A32
:101160001C121340964A9B009B580435FFF78EFAD9
:10117000A300FE1A04933B00083B1868FFF766F9CA
:101180003B1F04001868FFF761F9E217C30F8442A0
:1011900053419B003360049BFF1A8A4B04371B7832
:1011A000002B02D0019EFFF740FA2B68029A1C1216
:1011B0001340834A9B009B580435FFF767FA3B00B6
:1011C000083B1868FFF742F93B1F04901868FFF7C7
:1011D0003DF9049AA600BC1B0023824200DD0433C3
:1011E0002360784BBF1B1B780437002B02D0019E75
:1011F000FFF71BFA2B68029A1C121340704A9B00DF
:101200009B580435FFF742FA3B1F1B68A400043BC0
:10121000591E8B413A1B17009B001360694B043722
:101220001B78002B02D0019EFFF7FFF92B68029A72
:101230001C121340624A9B009B580435FFF726FAA4
:10124000A300FC1A04933B00083B1868FFF7FEF864
:101250003B1F06001868FFF7F9F836180120049BB9
:101260007600FF1A574B06431B7826600437002B85
:1012700002D0019EFFF7D9F92B68029A1C12134085
:101280004F4A9B009B580435FFF700FAA300FE1A53
:1012900004933B00083B1868FFF7D8F83B1F040095
:1012A0001868FFF7D3F8241A0120049B6400FF1A82
:1012B000444B04431B7834600437002B02D0019E5A
:1012C000FFF7B3F92B68029A1C1213403C4A9B00AB
:1012D0009B580435FFF7DAF9A300FC1A04933B008E
:1012E000083B1868FFF7B2F83B1F06001868FFF7C5
:1012F000ADF846430120049B7600FF1A314B0643AC
:101300001B7826600437002B02D0019EFFF78DF971
:101310002B68029A1C121340294A9B009B580435E3
:10132000FFF7B4F93B00083B1868FFF78FF83B1F45
:1013300004901868FFF78AF80100049805F0B8FCDB
:101340000123A4003E1B3700400018431D4B3060B2
:101350001B780437002B02D0019EFFF766F92B683B
:10136000029A1C121340164A9B009B580435FFF743
:101370008DF93B00083B1868FFF768F83B1F0490A5
:101380001868FFF763F80100049805F077FD012362
:10139000A4003E1B3700490019430A4B31601B78FB
:1013A0000437002B02D0019EFFF73FF92B68029A09
:1013B0001C121340024A9B009B580435FFF766F944
:1013C000789E00005C0200203B1F1868FFF73EF883
:1013D000C317C01858400123A4003E1B370040002B
:1013E0001843EA4B30601B780437002B02D0019E73
:1013F000FFF71BF92B68029A1C121340E44A9B006A
:101400009B580435FFF742F9A300FE1A0793306892
:10141000012C03D1FFF71AF8049008E0FFF716F843
:1014200004007068FFF712F80130031B0493049B5B
:10143000002B01DC0123049307F0EEFD049905F075
:101440001DFD0C190121079B6400FF1ACF4B0C43B3
:101450001B7834600437002B02D0019EFFF7E5F8BB
:101460002B68029A1C121340C94A9B009B580435F2
:10147000FFF70CF9A4003E1B3000FEF7BDFF37005C
:10148000C24B30601B780437002B02D0019EFFF75F
:10149000CCF82B68029A1C121340BD4A9B009B5843
:1014A0000435FFF7F3F8A300FE1A04933B00083B52
:1014B0001868FEF7CBFF3B1F04001868FEF7C6FF55
:1014C00004400120049B6400FF1AB04B04431B78C6
:1014D00034600437002B02D0019EFFF7A6F82B687A
:1014E000029A1C121340AA4A9B009B580435FFF72E
:1014F000CDF8A300FC1A04933B00083B1868FEF7E4
:10150000A5FF3B1F06001868FEF7A0FF0643012059
:10151000049B7600FF1A9D4B06431B782660043718
:10152000002B02D0019EFFF780F82B68029A1C1254
:101530001340974A9B009B580435FFF7A7F8A30078
:10154000FC1A04933B00083B1868FEF77FFF3B1F23
:1015500006001868FEF77AFF46400120049B7600DB
:10156000FF1A8A4B06431B7826600437002B02D0F3
:10157000019EFFF75AF82B68029A1C121340844A06
:101580009B009B580435FFF781F83B1F1868FEF756
:101590005DFFC0430123A4003E1B370040001843F9
:1015A0007A4B30601B780437002B02D0019EFFF786
:1015B0003CF82B68029A1C121340754A9B009B58FA
:1015C0000435FFF763F8A300FE1A04933B00083BC1
:1015D0001868FEF73BFF3B1F04001868FEF736FF54
:1015E0008440012364001C43049B3460FF1A674B52
:1015F00004371B78002B02D0019EFFF716F82B68EA
:10160000029A1C121340624A9B009B580435FFF754
:101610003DF8A300FE1A04933B00083B1868FEF750
:1016200015FF3B1F04001868FEF710FF044101235B
:1016300064001C43049B3460FF1A544B04371B782E
:10164000002B02D0019EFEF7F0FF2B68029A1C12BD
:1016500013404F4A9B009B580435FFF717F83B0097
:101660000C3B1868FEF7F2FE3B00083B06001868CA
:10167000FEF7ECFEF1170200C317300005F050FC36
:101680003B1F049005911868FEF7E0FE02000498E5
:10169000059905F0F9FB0123A4003E1B370040002B
:1016A00018433A4B30601B780437002B02D0019E60
:1016B000FEF7BBFF2B68029A1C121340344A9B00B2
:1016C0009B580435FEF7E2FFA4003E1B3000FEF7F6
:1016D000AEFD37002D4B30601B780437002B02D055
:1016E000019EFEF7A2FF2B68029A1C121340284AA3
:1016F0009B009B580435FEF7C9FFA4003E1B300039
:10170000FEF7A5FD3700214B30601B780437002B16
:1017100002D0019EFEF789FF2B68029A1C1213402B
:101720001B4A9B009B580435FEF7B0FFA4003F1BEB
:101730003800FEF79EFD154B1B78002B02D0019E52
:10174000FEF773FF2B68029A1C121340104A9B008D
:101750009B580435FEF79AFFA4003E1B3000FEF7AD
:10176000BAFD3700094B30601B780437002B02D0DC
:10177000019EFEF75AFF2B68029A1C121340044A7E
:101780009B009B580435FEF781FFC0465C02002099
:10179000789E0000A4003F1B3800FEF7D3FDE64B07
:1017A0001B78002B02D0019EFEF73FFF2B68029AA8
:1017B0001C121340E14A9B009B580435FEF766FF5C
:1017C000A4003E1B3000FEF7F7FD3700DA4B306017
:1017D0001B780437002B02D0019EFEF726FF2B68F2
:1017E000029A1C121340D54A9B009B580435FEF701
:1017F0004DFF069A3B1D0493CF4C9B1ADB2B04DD57
:101800001A23019E2370FEF710FF02F001F9012355
:101810004000184323783860002B03D0019E049FBA
:10182000FEF703FF2B68029A1C121340C34A9B0069
:101830009B58049F0435FEF729FF069A3B1D04932D
:10184000BD4C9B1ADB2B04DD1A23019E2370FEF78F
:10185000ECFE02F0D3F8BA4B4000184001231843C5
:1018600023783860002B03D0019E049FFEF7DDFE35
:101870002B68029A1C121340B04A9B009B58049F8D
:101880000435FEF703FFA300FB1A04930123200095
:101890001A000499FEF712FEAA4C2068643001F089
:1018A000FBFB002816D0039B21685A78A64801F05C
:1018B00072FE15E0A300FB1A04932000012300220E
:1018C0000499FEF7FBFD9F4C2068643001F0E4FBB7
:1018D000002802D1043DFEF7BCFE9B4801F0F6FC57
:1018E0000123039A137002F089F8C8222368D200FA
:1018F000063353431818039B5860FEF7ABFEA40051
:101900003E1BFEF753FE37008B4B30601B780437CD
:10191000002B02D0019EFEF788FE2B68029A1C1253
:101920001340864A9B009B580435FEF7AFFEA40087
:101930003E1B300002F0A0F837007F4B30601B7870
:101940000437002B02D0019EFEF76FFE2B68029A2F
:101950001C121340794A9B009B580435FEF796FEF3
:10196000A4003E1B300002F089F83700724B306053
:101970001B780437002B02D0019EFEF756FE2B6821
:10198000029A1C1213406D4A9B009B580435FEF7C7
:101990007DFEA4003E1B300002F072F83700664B5B
:1019A00030601B780437002B02D0019EFEF73DFE0D
:1019B0002B68029A1C121340604A9B009B58043506
:1019C000FEF764FEA4003F1B380002F077F85A4B84
:1019D0001B78002B02D0019EFEF727FE2B68029A8F
:1019E0001C121340554A9B009B580435FEF74EFECF
:1019F000A300FE1A31002000049302F081F8049B3A
:101A00003060FF1A4C4B04371B78002B02D0019E2C
:101A1000FEF70BFE2B68029A1C121340474A9B00EC
:101A20009B580435FEF732FEA4003F1B380002F03D
:101A3000A1F8414B1B78002B02D0019EFEF7F5FD6B
:101A40002B68029A1C1213403C4A9B009B58043599
:101A5000FEF71CFE0121200002F074F8364B1B78C3
:101A6000002B02D0019EFEF7E0FD2B68029A1C12AB
:101A70001340324A9B009B580435FEF707FE0021B5
:101A8000200002F05FF82C4B1B78002B02D0019E47
:101A9000FEF7CBFD2B68029A1C121340274A9B00CD
:101AA0009B580435FEF7F2FDA4003E1B300002F007
:101AB0007FF83700204B30601B780437002B02D0B2
:101AC000019EFEF7B2FD2B68029A1C1213401B4ABE
:101AD0009B009B580435FEF7D9FDA4003E1B300047
:101AE00002F07AF83700144B30601B780437002B73
:101AF00002D0019EFEF799FD2B68029A1C1213403A
:101B00000E4A9B009B580435FEF7C0FDA4003F1B06
:101B1000380002F03BF8084B1B78002B02D0019EE6
:101B2000FEF783FD2B68029A1C121340034A9B00A8
:101B30009B580435FEF7AAFD5C020020789E000049
:101B4000FEFFFF7F6402002068020020A4003F1B0C
:101B5000380002F077FDD94B1B78002B02D0019E94
:101B6000FEF763FD2B68029A1C121340D44A9B00B7
:101B70009B580435FEF78AFDA4003E1B300002F09E
:101B8000F5FD3700CD4B30601B780437002B02D0B9
:101B9000019EFEF74AFD2B68029A1C121340C84AA8
:101BA0009B009B580435FEF771FDA4003F1B3800D5
:101BB00002F0F8FCC14B1B78002B02D0019EFEF70F
:101BC00034FD2B68029A1C121340BD4A9B009B589F
:101BD0000435FEF75BFDA4003E1B300002F0F8FC6C
:101BE0003700B64B30601B780437002B02D0019EC3
:101BF000FEF71BFD2B68029A1C121340B04A9B0093
:101C00009B580435FEF742FDA4003F1B380002F04C
:101C1000D9FAAA4B1B78002B02D0019EFEF705FDD6
:101C20002B68029A1C121340A54A9B009B5804354E
:101C3000FEF72CFDA4003F1B380002F0D9FA9F4BA1
:101C40001B78002B02D0019EFEF7EFFC2B68029A56
:101C50001C1213409A4A9B009B580435FEF716FD50
:101C6000A4003F1B380002F0D3FA944B1B78002BE2
:101C700002D0019EFEF7D9FC2B68029A1C12134079
:101C80008F4A9B009B580435FEF700FDA4003F1BC4
:101C9000380002F0E5FA894B1B78002B02D0019E38
:101CA000FEF7C3FC2B68029A1C121340844A9B0067
:101CB0009B580435FEF7EAFCA300FE1A3100200011
:101CC000049302F0DDFD049B3060FF1A7B4B043768
:101CD0001B78002B02D0019EFEF7A7FC2B68029A0E
:101CE0001C121340764A9B009B580435FEF7CEFC2D
:101CF000A300FE1A31002000049302F0C9FD049BEA
:101D00003060FF1A6D4B04371B78002B02D0019E08
:101D1000FEF78BFC2B68029A1C121340684A9B004A
:101D20009B580435FEF7B2FCA300FE1A31002000D8
:101D3000049302F0B5FD049B3060FF1A5F4B04373B
:101D40001B78002B02D0019EFEF76FFC2B68029AD5
:101D50001C1213405A4A9B009B580435FEF796FC10
:101D6000A300FE1A31002000049302F0D3FB049B71
:101D70003060FF1A514B04371B78002B02D0019EB4
:101D8000FEF753FC2B68029A1C1213404C4A9B002E
:101D90009B580435FEF77AFCA4003F1B380002F084
:101DA00087FA464B1B78002B02D0019EFEF73DFCC4
:101DB0002B68029A1C121340414A9B009B58043521
:101DC000FEF764FCA300FF1A3900200002F022FB9A
:101DD0003A4B1B78002B02D0019EFEF726FC2B68A5
:101DE000029A1C121340364A9B009B580435FEF79A
:101DF0004DFCA4003E1B300002F0D8FA37002F4BF8
:101E000030601B780437002B02D0019EFEF70DFCDA
:101E10002B68029A1C121340294A9B009B580435D8
:101E2000FEF734FCA300FF1A3900200002F0A0FAEC
:101E3000224B1B78002B02D0019EFEF7F6FB2B688D
:101E4000029A1C1213401E4A9B009B580435FEF751
:101E50001DFCA300FF1A3900200001F09FF8174B6A
:101E60001B78002B02D0019EFEF7DFFB2B68029A45
:101E70001C121340124A9B009B580435FEF706FCC7
:101E8000A300FE1A31002000049301F087F8049BA0
:101E90003060FF1A094B04371B78002B02D0019EDB
:101EA000FEF7C3FB2B68029A1C121340044A9B00E6
:101EB0009B580435FEF7EAFB09B0F0BD5C02002038
:101EC000789E00000023F7B55A1E0192002B07DA16
:101ED00002F024F801F0D0FA01F082FB64230193B0
:101EE00000263000194B19688E4201DB019BEBE79D
:101EF000174B1A680132914200DC0022F0241A606C
:101F00001D68144F6C43E35D002B1DD0E419022BB8
:101F100016D0012B0ED1002801D101F06FFDF02267
:101F20006A430C4B0C499B185B68C31A8B4201D85F
:101F30000223BB54F0235D43064BEB5C022B03D121
:101F40002000FEF74BFBD1E70136CBE76002002013
:101F500000000020001200209F860100054B012197
:101F60001A68054B1A600023044AD1500433642BCD
:101F7000FBD17047B4050020AC0500205823002099
:101F800000B59BB00200054901A807F0C5F801A8FB
:101F900001F0B8F901F024FBFCE7C046B8A000004E
:101FA00037B5174D04002868002801D006F0A8FCBA
:101FB000A400200006F09AFC2860002801D11148F6
:101FC00009E001AB984208D20F4B02196B44019310
:101FD000934202D20D48FFF7D3FF042802D80830FD
:101FE0002860083C2B680A4A1C191360094B012120
:101FF0001C600023084AD1500433642BFBD137BD49
:10200000B4050020C9A000001CFCFFFFF9A00000DF
:10201000AC050020B00500205823002070B50D4D00
:102020000D4E2B684C1CA40036681C19B44203D911
:102030000A20FEF7B5FA0BE02C601D00AC4201D976
:1020400004C5FBE70F22090110400843186018007F
:1020500070BDC046AC050020B00500200322CB1C9B
:1020600070B50C00D9171140C9180500891000225D
:102070000420FFF7D3FF0023A34204DAE95CC2186F
:1020800011710133F8E7E1430023C91721404118DA
:102090000B7170BD10B5830706D1042804D90F2336
:1020A00004C81340042B03D00E20FEF779FA014830
:1020B00010BDC04609A2000070B501240B680D00D8
:1020C0001C4001D05C1002E00D20FEF769FA2000F0
:1020D00005F066F8264904F04FFF06F029FB02F0F0
:1020E0003DFF0022234B05F0DDFC0023002204F01D
:1020F0000DFF01242B681C40002819D0002C01D0B2
:102100005C1002E00D20FEF74BFA200005F048F8C5
:10211000174904F031FF06F00BFB02F01FFF00220D
:10212000144B05F0BFFC0022134B05F081F818E0BA
:10213000002C01D05C1002E00D20FEF731FA2000E7
:1021400005F02EF80A4904F017FF06F0F1FA02F044
:1021500005FF0022074B05F0A5FC0022064B05F009
:102160001BFF06F06DFA01234000184370BDC04606
:10217000D30237390000D0400000E03F10B5034AD9
:102180000121034800F0F6FE10BDC0460400002007
:1021900064A1000030B502248025094B094AED00F6
:1021A0009C505C59002CFCD0A124E400884204D24D
:1021B0008025ED0018514019F8E70021995030BDF5
:1021C00000E001400405000010B5002804D1E02023
:1021D0009C210002890203E09C2080218002C90228
:1021E000FFF7D8FF10BD002802D09C239B0201E01E
:1021F000E0231B021B6800201A0E532A01D11B0288
:10220000180A704730B501248025064A064BED00B8
:10221000D4505459002CFCD001600021014AD15007
:1022200030BDC04600E001400405000010B50028A4
:1022300002D09C20800201E0E0200002A6230902D7
:10224000DB05090A1943FFF7DDFF10BDF0B50124D6
:10225000802503000F4F08000F49ED007C507C598A
:10226000002CFCD09C46002810DD5478167893781A
:10227000240234431B0423431C00D37801381B067B
:102280002343644608C40432A446ECE700237B5091
:10229000F0BDC04600E001400405000070B5050037
:1022A0004B680A009C1C2100FFF7D0FFA0002818F3
:1022B00070BD0000154B1B68002B04D080219C23AF
:1022C000C9029B0203E09C21E02389021B02002833
:1022D00007D1191D5B6802001B0E522B14D10A0096
:1022E00012E0002281420FD903681B0E522B0BD142
:1022F000436802339B00C318994205D91A68110E2E
:102300000022522900D11A0010007047B80700209F
:102310008022F0B5520085B00021624806F003FB30
:10232000802200215200604806F0FDFA5F4B1B68D6
:102330001A00029353425A4110000392FFF744FFE0
:10234000029B002B01D15A4C00E05A4C0020FFF7B1
:10235000B1FFFF270500002D00D194E02B681A1271
:102360001B143A403B4001921A000A3A092A43D80A
:102370004C4B019A995C002900D07FE010224E4816
:1023800006F0D1FA2E00336801991A123A409142B0
:1023900017D11A143A400B2A06D0132A0CD00A2A55
:1023A0000FD1454B1E600CE03B40022B09DC424A3A
:1023B0009B00D3185E6004E0102200213E4806F026
:1023C000B2FA3000FFF776FF061EDCD13A4B1968EF
:1023D00000290FD02000FFF761FF0400374E31685D
:1023E000002903D02000FFF759FF0400344B0436C6
:1023F000B342F4D12B4B3EE0143B092B3ED82A4B81
:10240000019A995C002939D108222E4806F08BFAEE
:102410002E0033681A143A40152A0BD01D2A11D009
:10242000142A14D1019A1B123B409A420FD1254B1A
:102430001E600CE0019A1B123B409A4207D1214BCF
:102440005E6004E0082200211E4806F06CFA3000AD
:10245000FFF730FF061EDCD11A4E3168002909D083
:102460002000FFF71BFF71680400002902D0FFF76E
:1024700015FF04000C4B0121019A99542800FFF725
:1024800019FF050067E70298FFF7ADFE411C0398AE
:10249000FFF7CCFE054B039A1A600B4B1C6005B08E
:1024A000F0BDC046B8060020B8050020B8070020DF
:1024B0000470020004E00000BC230020C0230020C0
:1024C000CC230020CC230020BC07002070B50020C6
:1024D000FFF789FE04000120FFF785FE844200DA41
:1024E00004000A4B1E687542754128001D60FFF705
:1024F0006BFE002E01D0064B00E0064B064A28007A
:10250000611C1360FFF792FE70BDC046B807002043
:1025100004E0000004700200BC070020F8B50020B1
:10252000FFF761FE07000120FFF75DFE3E00224D30
:102530000643224C0CD18021E020C9020002FFF7A3
:1025400029FE01213000FFF771FE2E601C4B2FE0A9
:10255000874208DD00239C212B60194B89022360F0
:102560002368002011E0012380212B60154BC90254
:102570002360F5E71A68551C18D0120E522A07D1AD
:1025800001205A68023292009B188B42F2D311E06C
:10259000002800D023600C4C0C49200006F0E8FD18
:1025A000200001F03DFAFFF791FF04E0002802D07F
:1025B000236000E02160F8BDB8070020BC070020C0
:1025C00004E0000004700200102400207AA1000042
:1025D000F0B585B0039203220333DC1714402A4E72
:1025E000E3189C10336801900291002B02D08022E6
:1025F000D20201E09C229202244FA51C3B68AD0050
:102600005B199A4217D2FFF783FE3368002B02D082
:102610008022D20201E09C2292023B685B199A421E
:1026200009D21B4C1B49200006F0A2FD200001F03E
:10263000F7F9002026E0029B3E681B06190C6B464A
:102640001A7BA423DB051343019A0B431104FF22D9
:102650001204114019433000FFF7D4FD3300301D40
:102660000833210001933B60FFF7CCFD002C04D020
:102670000A9A21000198FFF7E9FD3000019B083D0F
:102680005D193D6005B0F0BDB8070020BC07002013
:1026900010240020A3A1000070B59AB0FFF73EFF00
:1026A000FF221F4CD2000021200006F03CF9002040
:1026B000FFF700FEFF25002600281AD003681A1431
:1026C0002A400A2A08D11A122A40FF2A0ED0D20024
:1026D000A1180B71A05009E0132A07D11B122B403F
:1026E000FF2B03D0DB00E2181671E650FFF7E2FD86
:1026F000E2E7FF210200C900235808305D1EAB410C
:10270000D2188842F8D1074901A806F005FD01A8B2
:1027100000F0F8FD044800F0F5FD1AB070BDC046A9
:10272000601B0020CAA10000E2A1000000220121DC
:10273000094B5A60094A51605A68002AFCD00022AD
:10274000C021054B49001A61044B01329A60044BC9
:1027500001325A501A607047FC10004000100040CF
:1027600000E100E00222064B0121DA670022054B5E
:102770005A61054A11615A69002AFCD07047C04667
:1027800004E100E0FC1000400010004010B5054BD3
:102790001A781C00002A01D0FFF7E4FF0023237001
:1027A00010BDC04648080020024B186801234000B5
:1027B000184370474408002000487047EC2300206D
:1027C000024B186801234000184370477C0000202A
:1027D00070B504000D00160001F01AF980230122E3
:1027E00000215B055B6E6270E270020AA271020C4E
:1027F000E2711A0A60716372000EA2721A0C1B0E4B
:10280000267025712072A170E272237370BD0000E2
:10281000124B10B51B68124C5A1C0FD0114C002BD8
:102820000CD0114C012B09D0104C022B06D00D4CB2
:10283000042B03D00E4C052B00D10B4C21000D486E
:1028400006F096FC200006F09BFC030004220433F3
:102850009B0809481B011343036010BD8000002042
:10286000ACA20000A5A20000B7A20000BCA200001C
:10287000B1A20000D8230020D423002070B5214C41
:102880002278002A3DD1204B01215A608022D205B6
:1028900011605A68002AFCD0002207201B4B1C49FB
:1028A00001255A500439585008315A5019481A49CC
:1028B00058501A491A485A501A495A50A622D2005A
:1028C0009D50082218495A50043158500220174987
:1028D000585017481749585017480439585018206D
:1028E00016495850C12189005A500539FF395A58A4
:1028F000083802435A50124A12499950FFF716FFFE
:10290000257070BD48080020FC0000400010004009
:102910000C050000746962751C05000024050000A8
:10292000200004022C0500001405000034050000FE
:10293000FFFF00003C0500002110010054050000CD
:1029400004050000C007002010B500280EDD0C684B
:10295000E3070BD56410FF2C08D8054B1B78002B20
:1029600001D1FFF78BFF034B034AD45010BDC04683
:1029700048080020240500000010004013B500287E
:1029800015DD0C68E30712D5082209496846641072
:1029900005F0C0FF072C0AD8064B1B78002B01D18D
:1029A000FFF76CFF6B46044A1957044BD15016BD14
:1029B0009DA2000048080020001000400C05000007
:1029C00010B5002813DD0C68E30710D56410532CF4
:1029D0000DD8074B1B78002B01D1FFF74FFFFFF7F6
:1029E000C1FEA123034ADB00D450FFF79FFE10BDB8
:1029F000480800200010004070B50E4B06001B7800
:102A0000002B01D1FFF73AFF00200B4D2C788442B8
:102A10000ED00A4B202219780323091B1940084BBA
:102A200049015918300005F075FF0120013C2C7058
:102A300070BDC0464808002049080020400800201A
:102A4000C0070020002330B589B0984226DD03245A
:102A50000D682C409C4221D12300042D1ED90F214A
:102A60002A681140062919D112091F2A16D9684669
:102A7000FFF7C2FF2300002810D06B460120197811
:102A80000123A14203DB6B461B5D5B000343A200F5
:102A9000AA1801345360202CF2D10423180009B085
:102AA00030BD0000F0B5424B8BB01B78002B01D13C
:102AB000FFF7E4FE02AD2800FFF79EFF002870D06C
:102AC0002B780B2B6DDD6B78012B6AD1EA78002314
:102AD000012A66D1374F384C3B6023712B79374A36
:102AE0001360002B0ED115256D446A782878AB78D9
:102AF000120202431B0413431A00EB781B06134314
:102B00003B6050E0012B10D115266E44727830786E
:102B1000B378120202431B0413431A00F3781A26F7
:102B20001B0613433B606A7C25E0022B02D16A7BC3
:102B3000162620E0042B0DD1152108226944684691
:102B400005F0E8FE0098019902F066F905F078FDBD
:102B5000386028E0052B26D11521082269446846F3
:102B600005F0D8FE0098019902F056F905F068FDCD
:102B70001E2638606A7D6E44132A00DD132200236E
:102B8000934204D0F05CE11808710133F8E70420A7
:102B90000021E21804339B101B01034311712360D1
:102BA00003E0002001E00022E9E70BB0F0BDC046E1
:102BB0004808002044080020EC230020800000206A
:102BC00010B5041E26D0144B1B78002B01D1FFF743
:102BD00055FEFFF7C7FD00201049114A114B8C50DC
:102BE00058600130086059680029FCD000200D4968
:102BF00008610A490130886019690029FCD00A4B34
:102C00000A491B785B01CB1804498B50FFF7AAFDDA
:102C1000FFF78CFD10BDC0464808002000100040A2
:102C200004050000FC10004040080020C007002000
:102C300030B589B000281EDD03230A6813401AD17D
:102C4000042A18D90F2011680840062813D1090951
:102C50001F2910D901240133990051580020214225
:102C600001D04910C8B26D46591E6854202BF2D1CC
:102C70006846FFF7A5FF09B030BD30B589B0002820
:102C800026DD0868830723D1042821D90F23026891
:102C90001340042B1CD1FFF7FDF9050006F070FA74
:102CA000041E122C00DD1224220002210D3268467F
:102CB000FFF78EFD6B465C730023A34205DA1A0012
:102CC000E95C6A4491730133F7E76846FFF778FFE0
:102CD00009B030BD70B50C0088B0012833DD08683C
:102CE000830730D104282ED90F2302681340042B08
:102CF00029D14B68DB0726D5FFF7CCF9060006F093
:102D00003FFA6468050064100E2800DD0E252A00D5
:102D1000012111326846FFF75BFD6B466A465C7322
:102D2000231293732314D3730023240E1474557445
:102D3000AB4205DA1A00F15C6A4491740133F7E79B
:102D40006846FFF73DFF08B070BD30B589B0002878
:102D500014DD0C68E30711D5102200216846FFF747
:102D600037FD6B466A4665105D73684663122D0E2B
:102D700064149373D4731574FFF722FF09B030BD48
:102D8000184B10B55A681849002A03D000225A601F
:102D900001328A601B691448002B22D00023114A9B
:102DA00013618022D2008458104A012C16D1A92325
:102DB000DB00C3585B4213600D4A1378032B01D824
:102DC0000133137003220B480378013313400A4A7E
:102DD00003705B01D318094A8B5000E01360012394
:102DE0008B6010BDFC100040001000407C000020F3
:102DF0004908002040080020C0070020040500000A
:102E000010B5034A0E21034800F0B4F810BDC046C7
:102E10000C000020C3A20000044A05491368C854EE
:102E200001339B059B0D13607047C046500C00207A
:102E30004A080020114A70B51368114C984211DA03
:102E4000015D451CFA39012906D8AB4206DD21187F
:102E5000497801391F2901D92800EFE70100251A17
:102E6000461C02D10023136006E0665C6E540131FB
:102E70008B42FADC181A106070BDC046540C00205A
:102E80005C0C002010B500F0B9FD064B1A689042AA
:102E900001D200221A601B68C01A034B8342804192
:102EA000404210BD580C0020204E000010B5094CC7
:102EB000094A2368126893420BD0084AD05C00F09C
:102EC000E1FE002805D0236801339B059B0D23609C
:102ED000EDE710BD5C100020500C00204A080020D7
:102EE00010B50400064B074A1B6812689B1ADB43A7
:102EF0009B059B0DA34202DAFFF7D8FFF2E710BD56
:102F0000500C00205C100020F7B506000191151E42
:102F10002FD05768B800441C0630FFF7E1FFFB20B4
:102F2000FFF77AFF1C20FFF777FFF0B2FFF774FF7F
:102F3000E0B22412FFF770FFE0B2FFF76DFF6B46BF
:102F40001879FFF769FF0026BE4212DAB300EB18CA
:102F50009C680136E0B2FFF75FFF2012C0B2FFF7B6
:102F60005BFF2014C0B2FFF757FF200EFFF754FF9E
:102F7000EAE7F7BD70B5074D2C68092C08DC0C2377
:102F80006343054E01349851F31859609A602C60E0
:102F900070BDC0466010002074240020F0B589B0D8
:102FA00004900E0001284BDD284B0868029383072C
:102FB00009D1042807D90F2302681340042B02D13A
:102FC000FFF768F80290214B70680393830709D1DB
:102FD000042807D90F2302681340042B02D1FFF7FE
:102FE00059F8039000271A4B1A4D1B680593059B4F
:102FF0009F4225DA2B1F0299186806F0AFF80028C7
:103000001BD12B686C6806930190019B069A934232
:1030100013DA20680399079406F0A0F80834002812
:1030200007D131000498079B08315B680238984744
:1030300009E0019B01330193E7E701370C35D6E73F
:103040001B20FDF7ADFA09B0F0BDC04609A2000093
:10305000601000207824002010B501F04FFA00F035
:10306000D1FDFFF78BF800F041FEFFF7C9FE01F03C
:10307000BDFA01F073FC10BD962210B512010021BB
:10308000034805F050FC0022024B1A6010BDC046F8
:103090000012002060020020064B074A1B681268DD
:1030A0009B1ADB439B059B0D0122834200DC00221F
:1030B00010007047500C00205C100020F8B505008F
:1030C0000C0016001F1E0ED10320FFF7E5FF00289D
:1030D00027D0FA20FFF7A0FEE8B2FFF79DFEE0B28E
:1030E000FFF79AFE1DE0501DFFF7D6FF002818D00D
:1030F000FB20FFF791FEE8B2FFF78EFEE0B2FFF78C
:103100008BFEF0B2FFF788FE3012C0B2FFF784FEEC
:103110003C00E31B9E4204DD2078FFF77DFE013476
:10312000F7E7F8BD70B50024F0250B4B1B689C42F7
:103130000EDA2A006243094BD3181A78002A05D008
:103140005978002311201A00FFF7B8FF0134ECE78B
:10315000FFF792FF70BDC046600200200012002001
:103160000123F3B50400FFB00D0010001A420DD08A
:1031700002AA1370431002A9537042121B0E40148E
:103180008A700B71C8700B00052273E00323134093
:103190001ED1042A1CD90F2201680A40042A17D123
:1031A000023302AA1370FEF775FF060005F0E8FF70
:1031B000F823FF33984200DD18000023834205DA2C
:1031C00001335A1EB25C02A9CA54F7E7421C50E010
:1031D000042801D0002809D1032302AA043813705F
:1031E0004342434153701300022243E0002B45D178
:1031F000042843D90F2102681140052912D1043354
:1032000002A90B70F8231209FF3392009A4200DDE5
:103210001A00002393422BDA0133C118C97802AE99
:10322000F154F7E7062929D101390E001209564356
:103230000196F826019FFF36B7421FDC02AE3170BF
:103240000136934213DA012701339900415839427C
:1032500001D0394100E00A49012737700F1271701F
:10326000B7700F14090EF77031710536E9E7019A4E
:10327000013202AB29002000FFF720FF7FB0F3BD31
:1032800019FCFFFF70B5F023050000240D4A18005B
:10329000604380184178A94203D001340A2CF6D14A
:1032A0000FE0F022002105F03EFB074A1368013BC6
:1032B000A34200D11460002329001A001120FFF757
:1032C000FDFE70BD001200206002002010B5B2B0FB
:1032D00002236A460400137005F052FFC72800DD80
:1032E000C7200023834205DA694601335A1EA25CD7
:1032F000CA54F7E7421C6B46FE211420FFF7DEFE9E
:1033000032B010BD10B5B2B002236A46040013708B
:1033100005F036FFC72800DDC7200023834205DA09
:10332000694601335A1EA25CCA54F7E7421C6B4639
:10333000FF211420FFF7C2FE32B010BDF7B5234BBA
:1033400006001B68F020009300232149009A934255
:103350000ADA02005A438A185478B44202D1127829
:10336000002A31D10133F1E70024F0231A0062432F
:1033700001920199164A55182F78002F06D0013472
:103380000A2CF3D11348FFF7BDFF1DE0F0223900EE
:10339000280005F0C8FA02230D4A0199EB60535446
:1033A0000D4AF1008A58009B6E70AE70AA602F61C2
:1033B0006F61A34202DC054B01341C600023310025
:1033C0001A001020FFF77AFEF7BDC0466002002009
:1033D000001200207EA30000601B002010B5FFF744
:1033E000A1FE0024064BE200D3181B79043B012BFD
:1033F00002D8E0B2FFF7A2FF0134FF2CF2D110BDDA
:10340000601B0020F7B50E0000247F250190194BAA
:10341000E200D1180979062901D0032926D198584C
:1034200083682B401C2B21D1C3681A002A40042A30
:103430001CD102692A40192A18D11B0A01339B00AA
:103440000C30C018FEF726FE070005F099FE002399
:10345000B0420BD19E4206DD019AF95CD25C9142EA
:1034600004D10133F6E7E0B2FFF768FF0134FF2C27
:10347000CDD1F7BD601B002070B500F0BFFA184B2E
:103480001A68904201D200221A601A681549821AFD
:103490008A4223D91860002000F08AFB444244414C
:1034A000604207240443002000F096FB002810D05F
:1034B000082600250C4BEA00D3181B799C4201D04A
:1034C000B34202D1E8B2FFF739FF0135FF2DF1D148
:1034D00004E0631C02D001267642EAE770BDC046D4
:1034E0004C0C00200F270000601B002037B5002483
:1034F0000500FFF717FE01A8019400F047FB20002C
:1035000000F076FE00F00AFD00F07AFB00F079FB97
:1035100000F046FF00F09EFA0548FFF7F3FEA542D3
:1035200004D0FEF71BFD0348FFF7ECFE37BDC04695
:1035300093A30000ABA30000002310B501001A0004
:103540001120FFF7BBFD10BD07B56B46197069462A
:103550005A7013128B701314120ECB700A716B46D3
:10356000010005221320FFF7A9FD07BD10B50A00D1
:1035700001001220FFF7F4FD10BD70B50500080032
:103580000C003230FFF7ACFC2B00220000211B2086
:10359000FFF794FD70BD10B50C000300110014205E
:1035A0002200FFF78BFD10BD70B506000020FEF76E
:1035B00081FE0024FF25002810D003681A142A4039
:1035C000152A05D11B122B40B34204D1040002E09E
:1035D0001D2A00D10024FEF76DFEECE7200070BD2F
:1035E000F0B580279DB0FFF761FCB94DB94C286854
:1035F000FF00391A201800F02BFB2B680600C318B7
:103600002B60002B00D1DBE1002E0DDD2868391A7C
:10361000201800F01DFB2B6806001B182B6000F023
:10362000EDF9AD4B1860EFE72378FA2B00D00CE1F1
:103630002B68022B06DCFFF725FC002800D1BFE138
:103640000120B8E16078A5780238182800D9FAE09E
:1036500003F09AFA0D1E22262932F93D676F75890B
:10366000DAEFF9F9F9F9F9F9F9F9F9F9F300FF2DB8
:1036700000D1E8E02800FFF705FE00229749EB00A3
:103680005A50CB181A7129000092130013204DE0F4
:103690002800FFF753FED6E02800FFF7F3FDD2E045
:1036A000FFF79CFECFE0FFF73DFD0020FFF71EFF78
:1036B0008B48FFF727FEC6E0182D00D9C3E0894BE1
:1036C000AA00D25829001520FFF74AFDBBE00024CC
:1036D0002000FFF769FF071E03D10134192CF7D131
:1036E000B1E0083005F04CFD06000530FFF7F8FBAF
:1036F000FB20FFF791FB1D20FFF78EFBE0B2FFF7E9
:103700008BFBF0B2FFF788FB3012C0B2FFF784FBEF
:103710000025AE42E1DD7B19187AFFF77DFB01350C
:10372000F7E700211D200B000A000091FEF750FF73
:1037300089E000222900009213002720F6E700F01C
:1037400077F903AC684A64210090684B200005F0CB
:10375000B1FC02232000237005F012FD23000200BB
:10376000002116206DE000245C4AE300D558002DAE
:1037700046D06B689E00701DFFF7B2FB2B00002542
:103780003200083321000120FFF798FC0020FEF7EB
:1037900091FD2E002F0000281DD0FF2103681A1272
:1037A0000A40A24214D11A140A400B2A07D10B4036
:1037B0000DD0012B09D0022B00D1FFE008E0132A25
:1037C00006D100252E002F0002E0060000E00700D1
:1037D000FEF770FDDFE7002E04D03200012120004B
:1037E000FFF792FB002D04D02A0002212000FFF7F2
:1037F0008BFB002F04D03A0000212000FFF784FB50
:103800000134FF2CB0D11EE0FFF78CFC0025002412
:10381000290000942300220013200135FEF7D8FE72
:10382000FF2DF4D1FF222100D2002C4805F07BF8B7
:1038300009E00120FFF75AFE05E0002329001A00E5
:103840001A20FFF73BFC0320B5E0FB2B00D0F7E686
:103850002A68042A00DCEEE62679E078244B36025A
:1038600006439E4200DDEBE6331D9A4200DCE2E6B1
:10387000E35CFE2B00D0E3E66078A578731E1C287D
:1038800068D007D8082835D01B285ED0012800D082
:1038900090E007E01E2800D17EE066D31F2800D10B
:1038A00080E087E0FF2D00D184E02800FFF7EAFCEC
:1038B00067790634B31E290000943A000A20FEF707
:1038C00087FE064BED00E8505D192F7172E0C0468F
:1038D000540C00205C0C0020580C0020601B0020C1
:1038E000BBA3000058230020D2A30000CDA30000FA
:1038F000F6030000182D5DD86079022813D0032844
:103900001BD0012856D1A71D7A78A479BB78120262
:1039100022431B0413431A00FB78AD001B0613431C
:103920005B0003430EE0002B44DDB11EA01DFEF73B
:1039300095FB244BAD00E8503CE0A379AD005A1E46
:1039400093419B001F4AAB5034E0601D1900FFF704
:1039500059FD2FE0FF2D2DD06279022A2AD8063496
:10396000B31E009429000B2022E0632B00DD6323AB
:10397000002203A8934204DDA11849798154013241
:10398000F7E7D9430022C917194041180A700133DB
:103990000090290015200BE0053400940022290036
:1039A0001E2005E0042B05D10022290005340094D7
:1039B000FEF70EFE701DFFF73DFA01E0050007E778
:1039C0001DB0F0BD58230020002070470020704734
:1039D000002070470020704701220020054B064957
:1039E0001A6158500330043158508018083158502B
:1039F0001A60704700800040040500000122034B5C
:103A00001A64A822D20098587047C046008000402F
:103A100010B5FFF7F3FFFA21890003F0BFF810BDDE
:103A200010B50100014802F063FE10BD8C110020AA
:103A300000487047E4A3000070B5054E0400335CF5
:103A40000D008B4202D002F07BFD355570BDC046A3
:103A50006410002070B50024064D635D012B05D174
:103A60000021200002F06CFD0023635501341D2C61
:103A7000F2D170BD641000200D2070473B207047CC
:103A8000036870B55B100120052B12D8094A9B0012
:103A90009C58094D2B5D002B05D00021200002F021
:103AA0004FFD00232B55200002F0F4FB01234000C2
:103AB000184370BD14A400006410002070B50368A2
:103AC00045685C106D1004D40B4B9D4202DD1D0057
:103AD00000E000251C2C0DD8084E335D012B05D0CD
:103AE0000121200002F02CFD012333552900200084
:103AF00002F05EFC70BDC046FF03000064100020B1
:103B00000B6870B55D101C2D16D80024012804DD4B
:103B10004C68043C624262415400094E735D9C4211
:103B200004D02100280002F00BFD7455280002F09B
:103B30003BFD0423012800D00023180070BDC046BF
:103B40006410002070B504000D001C280ED8084E2B
:103B5000335C012B04D0012102F0F2FC0123335528
:103B6000290020004D1EA94102F008FD70BDC0468D
:103B700064100020436810B5191F4A424A4100688A
:103B800011004010FFF7DEFF10BD000037B5694699
:103B90000200064B684630CB30C11368042B02D1BB
:103BA00000F036FB01E000F05BFB37BDDCA300005A
:103BB00010B5084C6379002B05D00021052002F0D8
:103BC000BFFC00236371052002F0EEFC4342584124
:103BD000800010BD6410002010B5084CE37A002B63
:103BE00005D000210B2002F0ABFC0023E3720B2078
:103BF00002F0DAFC43425841800010BD64100020FE
:103C00007047704710B5034A04210348FFF7B2F923
:103C100010BDC04684000020D3A20000E12110B5F1
:103C20004902094802F0ABFDFFF7D6FE0A2002F078
:103C30002BFB0023FF21054A995401331D2BFBD197
:103C400000F0AEFB10BDC0468C11002064100020B7
:103C5000F8B50B4E070030000D0002F0CFFD041E3A
:103C6000AC4200DD2C003D00EB1B9C4205DD30002A
:103C700002F0CEFD28700135F6E72000F8BDC04601
:103C80008C11002010B50100014802F07FFD10BD2D
:103C90008C1100200020704710B51E20FCF780FC1E
:103CA00010BD10B51E20FCF77BFC10BD10B51E200A
:103CB000FCF776FC002010BD10B51E20FCF770FC50
:103CC000002010BD10B51E20FCF76AFC10BD10B519
:103CD0001E20FCF765FC10BD10B51E20FCF760FC33
:103CE00010BD10B51E20FCF75BFC10BD10B5034ADB
:103CF00009210348FFF73EF910BDC046A40000208B
:103D00002CA400000123034A1360034A1068984062
:103D1000184370478C10002094100020202800D9F0
:103D20000020084B8000C25801239340064A0749EF
:103D30001360074A1160074A07491160074A136078
:103D40007047C04618A900008810002008050050E0
:103D5000A41000209C1000200C05005018050050F5
:103D6000F0B5EFF310810123194083F31088134E4F
:103D7000134AB4461268013A9340124A1468124A30
:103D80001568124A002B15D0166803420BD0266026
:103D9000C046C046C046C046C046C046C046C046F3
:103DA00016682E6004E067463E601668084F3E6065
:103DB0005B08E7E781F31088F0BDC04608050050B6
:103DC000F4000020A41000209C1000208810002087
:103DD0000C05005030B585B001AD0C220649280015
:103DE00004F098FD0024285D01210134FFF724FE32
:103DF0000C2CF8D105B030BDB8A40000F0B53B4C98
:103E000085B0210003220C31684604F083FD2100B7
:103E100009220F3101A804F07DFDFFF7F9FD344BB5
:103E2000344CC0182368984201D2002323602568CF
:103E3000002D3ED12E006B4604339F5D01213800DA
:103E4000FFF7FAFD01360121380002F097FB092E39
:103E5000F1D100266B469F5D01213800FFF7ECFD94
:103E600001360021380002F089FB032EF2D1C82070
:103E700080000138C046C046C046C046C046C04665
:103E8000C046C046C046C046C046C046F1D100212B
:103E90000420FFF7D1FD00266B460021985D013616
:103EA000FFF7CAFD032EF7D1FFF7B2FD13302060F4
:103EB00019E0FFF7ADFD23680025984213D30420D5
:103EC00002F0E8F90C4B0D4EC01801D4306000E050
:103ED00035603068032102F0EBFE00230125084A1B
:103EE000306023601360280005B0F0BDB8A4000066
:103EF0001027000084100020C8FEFFFF941000204F
:103F00008C10002010B50124044001D0441002E0C0
:103F10000D20FCF745FB200010BD00007FB5A44E2E
:103F20003368002B0BD1A34A1268002A07D1A24B99
:103F30001B68002B00D139E1FFF760FF36E19F4D90
:103F40002A68002A2AD19C4A1268002A07D0FFF763
:103F500055FF002800D129E1FFF73CFF05E0954A15
:103F60001268002A01D1002BF6D1924B19681A0071
:103F7000002911D03468002C0ED101AD0C229049DB
:103F800028001C6004F0C6FC285D00210134FFF706
:103F900053FD0C2CF8D109E13368136000211A207D
:103FA00002F0ECFA00211B2002F0E8FA00211C20AC
:103FB00002F0E4FA2E68012E56D0022E00D19CE0C9
:103FC000002E00D0ECE0013631007A4C032023684B
:103FD000994302F0D3FA0420216801400B005942B2
:103FE000594102F0CBFA102123680A200B405942B4
:103FF000594102F0C3FA8021236809010B4059425C
:104000005941062002F0BAFA8021236809020B40C8
:1040100059425941072002F0B1FA80212368490230
:104020000B4059425941092002F0A8FA8021236827
:1040300089020B4059425941192002F09FFA802110
:104040002368C9020B4059425941182002F096FAE0
:10405000802321681B030B4059425941172002F06D
:104060008DFA31001A2099E00221524C1720236862
:104070000B405942594102F081FA08212368182067
:104080000B405942594102F079FA80212368C90056
:104090000B4059425941042002F070FA80212368F4
:1040A00049010B40594259410A2002F067FA802128
:1040B0002368C9010B4059425941032002F05EFABE
:1040C0008021236889030B4059425941092002F09D
:1040D00055FA802321681B040B405942594119208D
:1040E00002F04CFA3100062002F048FA31000720B5
:1040F00002F044FA31001B2050E020212D4C172003
:1041000023680B405942594102F038FA4021236894
:1041100018200B405942594102F030FA802123689F
:1041200019200B405942594102F028FA8021236896
:1041300049000B4059425941092002F01FFA8021E1
:10414000236889000B4059425941072002F016FAB2
:104150008021236889010B4059425941062002F011
:104160000DFA8021236849030B40594259410A2026
:1041700002F004FA80212368C9030B4059425941D7
:10418000032002F0FBF9802321685B040B405942B5
:104190005941042002F0F2F901211C2002F0EEF94D
:1041A0002B680321581C02F069FE29607FBDC046C0
:1041B00098100020901000208C100020A0100020EB
:1041C000B8A40000006810B5C30703D5FFF79AFE36
:1041D000054B1860054B1B68002B03D0024B186879
:1041E00000F0BAFB10BDC04698100020AC100020B3
:1041F0000022054B10B51A60044B1B68934201D096
:1042000000F0A8FB10BDC04698100020AC100020A4
:1042100070B505000068FFF775FE04006868FFF7D9
:1042200071FE631E0100042B14D8451E042D11D805
:1042300005226A43D318012215009D402B00064831
:1042400005682B430360054B1B68002B02D0200040
:1042500000F081FB70BDC04698100020AC1000201B
:1042600070B505000068FFF74DFE04006868FFF7B1
:1042700049FE631E0100042B14D8451E042D11D8DD
:1042800005226A43D31801229A40130006480268A7
:104290009A43064B02601B68002B03D000222000CB
:1042A00000F059FB70BDC04698100020AC100020F3
:1042B0002C4BF7B51B680400002B03D101204042B2
:1042C000FFF72CFD01262468344219D0FF22631029
:1042D000180212041040FF22611212020A40DBB2DF
:1042E00010431843204B1B68202B06D1B4401F4BB2
:1042F000A40EA400E35800021843FFF731FD30E09C
:10430000032525402DD1042C2BD90F2322681340DF
:10431000062B26D1FF27130901933F04019B9D42E1
:104320001FDAAB00E3185A68324218D05310180253
:104330003840FF2184460902501208406146DBB232
:1043400008431843084B1B68202B06D15200920EDD
:10435000064B9200D35800021843FFF701FD0135C8
:10436000DCE7F7BD88100020F4000020E4A4000082
:104370000B6810B50200D80701D5581001E00120E4
:1043800040421823012A03DD4A68042A00D1083379
:10439000024A1360FFF7C2FC10BDC046F4000020C3
:1043A000012010B54042FFF7B9FC10BD0068F8B518
:1043B000C30702D5FFF7A6FD0BE0830726D104282B
:1043C00024D90F2203681A40042A1FD11B091DD0CB
:1043D00000790300203B5E2B18D8052200205343B0
:1043E0000B4E9D18043AAB420CD0052110249F5D62
:1043F0003C4200D080180139520064100029F7D1E6
:104400000133F0E701234000184300E00120F8BD2C
:10441000E4A50000F0B5050085B008680C00FFF7C2
:1044200071FD0390022D08DD6068FFF76BFD07004A
:10443000A068FFF767FD040001E0012427000523C1
:104440006343053B0293012326000193231D9E42F3
:1044500034DC3D003B1D9D422BDC731E042B23D816
:104460006B1E042B20D8029B039A591E019B4919ED
:104470001A40204B0AD001228A4019680A431A6068
:104480001D4B01221B68002B0ED009E00120884043
:104490000100186888431860174B1B68002B03D075
:1044A0003100280000F057FA019B01355B000193B1
:1044B000D0E7029B013605330293C7E73D1D042D6B
:1044C00015D8012C13D126003300AB40094A1168DE
:1044D0009943094B11601B68002B04D0781D002202
:1044E000210000F038FA01340535062CECD105B076
:1044F000F0BDC04698100020AC10002010B5034A53
:1045000001210348FEF736FD10BDC046EC00002037
:10451000D0A400000122094B1A60094A1368002B3D
:10452000FCD00322074B1B68D8171040C01801238A
:1045300080100638400018437047C04600C0004055
:1045400000C1004008C500400120704710B5064C6E
:10455000200000F039FB0549200000F059FB012242
:10456000034B1A6010BDC046D0100020801A060010
:10457000A810002010B501210D20FFF75DFA0121E0
:104580000E20FFF759FA00210F20FFF755FA044CCF
:10459000200000F055FA1021200000F06DFA10BD47
:1045A000BC10002010B504680D20E30703D564108B
:1045B000FF2C03D91720FBF7F3FF06E0FFF7DAFF24
:1045C000E1B2024800F07AFA002010BDBC100020D1
:1045D00010B5FFF7CFFF0021034800F06FFA012369
:1045E0004000184310BDC046BC10002010B5034A5F
:1045F00007210348FEF7BEFC10BDC046FC000020AA
:10460000BFA700000D4B70B51B6804000E0015001D
:10461000002B01D1FFF79AFFE1B2094C200000F016
:104620007FFBF1B2200000F090FAE9B2200000F028
:104630008CFA200000F0DEFB70BDC046A810002000
:10464000D010002010B501240368234205D0416832
:10465000214202D08268224201D10D2004E058108C
:104660004910802803D91520FBF79AFF0BE0FF299A
:1046700001D91620F8E75210FF2A01D91720F3E7D5
:10468000FFF7C0FF002010BDF7B501242300A042B2
:1046900037DD0A68144234D01B4B55101B684C6838
:1046A000002B01D1FFF752FF0127184EE9B230006D
:1046B00000F036FB3C4205D03C413000E1B200F056
:1046C00044FA1AE00325254017D1042C15D90F23ED
:1046D00022681340062B10D113090193019B9D42C0
:1046E0000BDAAB00E3185968394204D04910C9B25B
:1046F000300000F02AFA0135F0E7300000F07AFBD4
:1047000000231800FEBDC046A8100020D0100020D5
:10471000144B70B51B6805000E00002B01D1FFF78C
:1047200015FF114CEDB22900200000F0F9FAF1B2AA
:10473000200000F00AFA0021200000F0FDFA002815
:1047400001D040420CE001222900200000F0E3FAF1
:10475000200000F0F0F90028FAD0200000F0F0F975
:1047600070BDC046A8100020D010002010B5012454
:104770000368234202D04168214201D10D2004E0A8
:1047800058104910802803D91520FBF709FF07E0CE
:10479000FF2901D91620F8E7FFF7BAFF40002043B0
:1047A00010BD0000002370B5344D0400EB560133FA
:1047B0002BD10D211D20FFF7ABFF5A2804D1012278
:1047C0002A212A703D380AE00F211920FFF7A0FFA7
:1047D000332807D102235F2220212B701A38FFF7DC
:1047E00011FF12E00D211E20FFF792FFC7280AD10A
:1047F000032300222A21A9382B70FFF703FF1B2275
:104800002A211E20EBE700232B700023EB56022BFE
:1048100006D0032B13D0012B26D121001D2010E040
:10482000012C04D129211920FFF772FF0DE0032C80
:1048300015D12B211920FFF76BFF043C05E0210067
:104840001E200124FFF764FF64427F2801DD013848
:10485000FF3803007F330ADA7F20404207E0052C4F
:1048600002D12D211920ECE70124002064426423A9
:104870007F21584302F01CFA604370BDF80000200D
:1048800010B50120FFF78EFF01234000184310BD33
:1048900010B50320FFF786FF01234000184310BD29
:1048A00010B50520FFF77EFF01234000184310BD1F
:1048B000F8B501263400B04236DD0F683E4233D0F1
:1048C0004D68AB0730D1042D2ED90F232A68134031
:1048D000062B29D1154B1B68002B01D1FFF736FEA3
:1048E0000024354204D12B681C09202C00D9202437
:1048F0000F4E7F10F9B22200300000F00CFAA70032
:10490000EF19AF420DD0300000F015F90028FAD0B1
:10491000300000F015F901234000184368600435A9
:10492000EFE70120640004432000F8BDA810002038
:10493000D0100020002070470020704700207047F2
:10494000002070470020704700207047002070470B
:1049500000207047704770477047000010B5034A49
:1049600008210348FEF706FB10BDC04634010020B5
:1049700000A8000010B5FFF751F9AF20C000FDF707
:104980000FFBFEF769FB0448FEF7BCFCFDF784FE55
:10499000FEF724FD10BDC04693A3000010B5FDF73F
:1049A00091FA10BD70B5002504AC24780573A942B6
:1049B00005D10A4B0A4A23210A4803F02BFF016064
:1049C0000949920052589B0002715B588371A30001
:1049D0005B58856043710223C37170BD83A80000DA
:1049E00046A8000091A8000018A90000037B002B36
:1049F00004D1437383730361013303737047000071
:104A00001FB50191A02100240068C900D2B2445012
:104A1000012A07D0A24203D0032A05D1042202E0D2
:104A2000022200E006221343034A8350034B019AFB
:104A3000C250012343501FBD54050000240500004F
:104A400010B50400FFF7D2FFA1222368A179D2009C
:104A500099506179064A2000995021790432995081
:104A6000044B19685A689B68FFF7CAFF10BDC0461F
:104A70000C050000B01000204BB2002B0CDB802393
:104A80003F290CD81F290CD80F290CD807290CD87E
:104A900003290CD81B060BE080239B0408E0DB04F1
:104AA00006E01B0504E05B0502E09B0500E0DB057A
:104AB0000168014A8B507047240500000368074ACB
:104AC00099501A00FC32D1680029FCD0A321C900FA
:104AD00058580023C0B2D3607047C0461C05000080
:104AE00007B58022074BD2051A6000229A60023275
:104AF0001A710F230C3200930349023B0348FFF75E
:104B000051FF07BDB010002000300040BC10002055
:104B1000F8B505000E0017000024BC4208D02B6831
:104B2000315D1B6828009847002801D00134F4E764
:104B30002000F8BD704710B51C3001F005FE10BD17
:104B400010B51C3001F0F2FD10BD70B5437E0D00B4
:104B5000002B05D06430040001F005FE002801D0D0
:104B6000002004E02000290001F0D1FD012070BDEB
:104B700010B51C3001F0EEFD10BD0000F7B501933B
:104B8000FA23002504009B0083600D4B4560083329
:104B900003601C300F00160001F0AEFD20006430F1
:104BA00001F0AAFD074AB600B35827616375019B5F
:104BB00020009B009B586576A576A375FEBDC04678
:104BC000F8A8000018A900000123A022C375837D66
:104BD0000C49C133FF33D2059B009950437DC1334B
:104BE000FF339B009950CC210369074A490499502F
:104BF0000521243A9950817D08329950417D034A1C
:104C0000995070470C060000240500000C050000B8
:104C1000A02302690020DB00D0500948814204D95A
:104C20000848814204D9CD2103E0CC21490401E0A8
:104C30008021C904044811500521D1507047C04655
:104C4000A086010090D0030024050000F7B5050000
:104C500000200C00019382425CD0161E402E00D929
:104C600040262F001C37380001F05CFDB1222B6973
:104C7000D20080219C50012289005A50A97E00292F
:104C800001D11A621A600024731E2A69A34206D158
:104C9000019B002B03D0802302219B00D1500123D4
:104CA00013621300FC33D968002902D1996A0029E4
:104CB000F9D0996A00290AD1D960A323DB00D15821
:104CC0003800C9B2013401F022FDA642DCD8019AB5
:104CD0002B69002A04D11A00FC32916A00290AD0FB
:104CE00001210022AA7659611900FC318868002848
:104CF000FCD08A6007E00121A976D961D16C002936
:104D0000FCD00021D164FC339A6A002A01D0002231
:104D10009A62E0B2FEBD10B50123FFF797FF10BD08
:104D20000300AC3310B504001970643001F0FAFCD4
:104D30000123637610BD0000F8B500220D000100CC
:104D40004276AC31036904000878B121C90058509B
:104D5000802189005A5001321A629A602600643616
:104D6000300001F0F1FC00280ED03000276901F07E
:104D7000DDFC1E4BF8502369FC331A6A002A0CD163
:104D80009A6A002AF9D008E02369002D0AD11A0096
:104D9000FC32916A002905D10EE09A6A002AF3D10B
:104DA0001A62DBE701225A611A00FC32916800297D
:104DB000FCD00021916006E00121D961D16C00296D
:104DC000FCD00021D1641A000020FC32916A81429B
:104DD0000BD0074990625A5802305A50824204D090
:104DE000043A534253410230C01AF8BD1C0500007A
:104DF000C404000010B50121FFF79EFF10BD0000A4
:104E000010B51323142202490248FFF7B7FE10BD64
:104E100000400040D0100020F0B5474680B4CB0FD2
:104E200098464A4C4B005B0D1E1982B007000A00E1
:104E3000132E35DC002E57DB454B040033411F0099
:104E40000F4007430D00002F24D05B081C000C40CE
:104E500020430027002807D0132E00D172E08022C3
:104E6000D202324199430A434346DE00394B1100D6
:104E70009E1934687568380022002B0002F0D8F9BA
:104E8000009001910098019922002B0003F084F812
:104E900004000D002000290002B004BC9046F0BDC3
:104EA000332E0CDD802304000D00DB009E42F1D187
:104EB00002000B0002F0BCF904000D00EAE7264CEA
:104EC0000D00A446012463446442DC40A4466146CC
:104ED00004000142DED049080142C5D08027FF0509
:104EE0001F4188430743BFE74B005B0803430400AF
:104EF0000D00002BCED00B031B0B03435A42134370
:104F000080221B0B120313404A0C52041343190056
:104F10004346104ADB00D3181C685D6822002B0052
:104F200002F086F9009001910098019922002B006F
:104F300003F032F842464B005B08D60733430400C7
:104F40001D00A7E780273F0689E7C04601FCFFFF59
:104F5000FFFF0F00A0A90000EDFBFFFF30B5214AC5
:104F60004B0087B05B0893421EDD1F4A934205DD6C
:104F700002000B0003F010F807B030BD02AA00F0E9
:104F800035F803231840049A059B01281ED00228F7
:104F900011D000281FD00298039900F02DFA802329
:104FA0001B069C466144E7E7002300220093002390
:104FB00000F088FFE0E7012402980399009400F0D4
:104FC00081FF80231B069C466144D5E70298039924
:104FD00000F012FAD0E7012402980399009400F03F
:104FE00071FFC9E7FB21E93FFFFFEF7FF0B54E46B8
:104FF00057464546E0B4DC4B4E0090B0170089465A
:1050000076089E4200DC81E0D84B9E4220DCD84AE4
:10501000002900DC89E1D74B02F0BEFFD54B04002C
:105020000D009E4200D18AE0D34AD44B02F0B4FF77
:1050300002000B0020003A607B60290002F0ACFF08
:10504000CD4ACE4B02F0A8FFB860F960012066E0BF
:10505000CB4B9E4200DC8DE0CA4B9E4265DCCA49C8
:1050600032158A46924453461B05F51A290004005E
:1050700003F0E6FA03F01AFB02000B0020002900FF
:105080000A920B9302F088FF0022C04B02F00AFD47
:105090000290039103F0D4FA03F008FB04000D0022
:1050A00002000B00029803990C940D9502F074FF16
:1050B0000022B64B02F0F6FC002200230E900F9166
:1050C00001F000FF002800D14CE100230022200065
:1050D000290001F0F7FE0222431E9841131AAC4A40
:1050E0003900019202220AA80092524600F09EFA6C
:1050F0004B46002B13DA8022120694467B6840420E
:1051000063447B60FB686344FB6008E002000B00C3
:105110003A607B60002200230020BA60FB6010B080
:105120001CBC90469946A246F0BD02000B0002F05E
:1051300033FFB860F960386079600020EFE7D32270
:105140008E4B520502F028FF924A934B04000D004B
:1051500002F022FF02000B0020003A607B60290071
:1051600002F01AFF8B4A8C4B02F016FFB860F96010
:105170000120D4E700F056FF884A894B04000D0057
:1051800002F090FC0022874B02F052F803F058FA2C
:10519000804603F08BFA764A764B0690079102F030
:1051A00081FC02000B002000290002F0F5FE734B89
:1051B00002900391069807996F4A02F073FC4346E8
:1051C00004000D00049405951F2B30DC013B764A4A
:1051D0009B009B589E422AD002000B000298039924
:1051E00002F0DAFE02000B0005000C003A607B6062
:1051F000029803992A00230002F0CEFE049A059B30
:1052000002F0CAFE06000B003200BA60FB604B469B
:105210004046002B00DB82E780231B069C4664444B
:1052200061443D607C60BE60F960404277E7049A6B
:10523000059B0298039902F0AFFE0B0002003A6052
:105240007B604B0036155B0D05000C00F31A102B2C
:10525000CEDD06980799D322484B520502F022FC76
:1052600004000D0002000B000298039902F094FE66
:1052700002000B00029803990892099302F08CFE39
:1052800022002B0002F088FE04000D00069807990A
:10529000404A414B02F006FC22002B0002F07CFE4B
:1052A00002000B00049005910898099902F074FE21
:1052B00002000B003A607B604B005B0DF61A0500A4
:1052C000089A099B0C0002920393312E90DD0698F8
:1052D0000799B822304B920502F0E4FB04000D0060
:1052E00002000B000298039902F056FE0A0001002A
:1052F00013000291039202000898099902F04CFEF3
:1053000022002B0002F048FE04000D0006980799C9
:10531000264A274B02F0C6FB22002B0002F03CFE7F
:1053200002000B000492059358E7124B01F080FF36
:10533000104B04000D009E423CD00F4A0F4B01F071
:1053400077FF02000B0020003A607B60290002F02A
:1053500023FE094A094B01F06BFFB860F960012098
:105360004042DCE60323BAE6FB21E93F7BD9024059
:1053700000004054FB21F93F3163621A61B4D03D13
:10538000FB213941FFFFEF7FEAFBFFFF0000704187
:1053900030AA00007370032E8A19A33B83C8C96D1D
:1053A000305FE43F0000E03FB0A90000C149202584
:1053B0009A837B39D3220D4B520501F039FF0C4AF9
:1053C0000C4B04000D0001F033FF02000B00200025
:1053D0003A607B60290002F0DFFD054A054B01F0D1
:1053E00027FFB860F9600120404298E661B4D03DE3
:1053F0007370032E8A19A33BF0B54F464646C0B4DE
:1054000087B000920193754B4F00814688467F0814
:105410009F4263DC03F014F9002800D1DAE04A4629
:1054200043464846414602F03DFB04000D006C4AED
:105430006C4B02F037FB6C4A6C4B01F0F9FE22001A
:105440002B0002F02FFB6A4A6A4B02F0A5FD2200F6
:105450002B0002F027FB684A684B01F0E9FE2200AE
:105460002B0002F01FFB664A664B02F095FD2200FE
:105470002B0002F017FB644A644B01F0D9FE2200B6
:105480002B0002F00FFB029003910022604B2000E2
:10549000290002F007FB029A039B06000F00200080
:1054A000290002F0FFFA009A019B04000D00484613
:1054B000414602F0F7FA02000B002000290002F03A
:1054C0006BFD02000B003000390002F065FD0200A8
:1054D0000B0000204F4902F05FFD70E002000B005E
:1054E00002F0E0FA04000D003D4A3E4B02F0DAFA09
:1054F0003D4A3E4B01F09CFE22002B0002F0D2FA06
:105500003B4A3C4B02F048FD22002B0002F0CAFA55
:10551000394A3A4B01F08CFE22002B0002F0C2FA0D
:10552000374A384B02F038FD22002B0002F0BAFA5D
:10553000354A364B01F07CFE2B00220002F0B2FA15
:10554000354B029003919F429FDD344B00229F42D6
:105550003ADC334900207B182E4916001F0002F068
:105560001BFD049005910022294B2000290002F028
:1055700099FA32003B0002F00FFD029A039B0600ED
:105580000F002000290002F08DFA009A019B040010
:105590000D004846414602F085FA02000B0020004B
:1055A000290002F0F9FC02000B003000390002F083
:1055B000F3FC02000B000498059902F0EDFC07B023
:1055C0000CBC90469946F0BD164B002604920593FC
:1055D000154FC8E700200F49F1E7C046FFFF3F3EE7
:1055E000D43888BEE9FAA8BDC4B1B4BD9EEE213E50
:1055F000AD529C804F7E923E9015CB19A001FA3E91
:105600007751C1166CC1563F4C5555555555A53F60
:105610000000E03F0000F03F3233D33F0000E93F9D
:105620000000E0FF0000E73F0000D23FF0B5564623
:105630004D4644465F46F0B48E4CA544099119008E
:105640001400A89A0B938C4B9200D2580B00029036
:10565000013BE01E18211D0016000892009301F086
:1056600027FBC3430200DB171A401300110001336C
:105670000E929A009B1ADB001B1906934C1B76199D
:1056800018D4A99BA5009C46361926AF654401365F
:1056900007E0286803F00AF8013403C70435B44270
:1056A00008D0002CF5DA00200021013403C70435AE
:1056B000B442F6D1089B002B01DA00F0F9FB76AB7F
:1056C00019008B4626AA9146089A0A930132D20005
:1056D0009344029A9A469046009BDB009944083313
:1056E0009844009B002B00DAB5E14C4600260027C9
:1056F000029D2268636803CD02F0D4F902000B001A
:105700003000390001F094FD083C06000F004545CB
:10571000EFD15346C0C39A4608239C46E144DA457C
:10572000DFD10899554A0B00944663449B0012A8A8
:1057300084461A000298624483460D920B9A043301
:10574000D200634493440F930591059A0A98D300BD
:1057500019000C938C46030063441E685F68002A9E
:1057600034DD12AB99461300454A804694466344A3
:10577000DB00984474AB9A460022424B300039005B
:1057800002F090F902F05CFF02F090FF00223E4B25
:1057900004000D0002F086F902000B003000390011
:1057A00002F0FAFB02F04CFF4B4601C39946434618
:1057B00020001A685B68290001F03AFD08235B426B
:1057C0009C46E04406000F00D045D5D1069B300032
:1057D0001A003900994600F0C1FCFF2300229B0506
:1057E00004000D0002F05EF900F020FC0022274BBF
:1057F00002F058F902000B002000290002F0CCFB57
:1058000004000D0002F01CFF804602F04FFF020072
:105810000B002000290002F0BFFB4C4606000F00E1
:10582000002C00DCF8E0059B18205A1E920012ABF9
:105830009B58001B19000141884481405B1A12A942
:105840008B501722121B13410793079B002B4BDD34
:1058500001239C46059BE044002B00DCF2E28025FE
:105860001096119712AB0021002409486D04059F82
:1058700019E0C04684FDFFFF38AB0000FEFFFF3F8C
:10588000FFFFFF1F0000703E00007041000020403D
:10589000FFFFFF00002A02D0AA1A1A60013401316A
:1058A00004338F4209DD1A68002CF3D0821A0131CB
:1058B0001A60012404338F42F5DC109E119F069B71
:1058C000002B0EDD012B00D1B1E0022B09D1059B8D
:1058D00012A95A1E920012AB9B5810939B029B0A6E
:1058E0008B50079B022B7ED0002300223000390012
:1058F00001F0E8FA059B002800D16BE208995A1ED6
:10590000914210DCBF490F988C4612A963448C4623
:1059100000219B0063441C68043B21438342FAD16D
:10592000002900D0B5E0089B12AA013B9B00D35888
:10593000002B00D084E201220D9B043B5968013208
:105940000029FAD005990B008C4601336244079276
:10595000934242DC0E9A9446A99A634492460B9A6B
:105960009B00944626AA90469A44059B0A9A634453
:10597000DB0098440C9B94469946079BE144DB006E
:10598000634405935346186802F090FE434618603E
:105990005960009B002B23DB444600260027029D14
:1059A0002268636803CD02F07DF802000B0030002E
:1059B000390001F03DFC083C06000F005D45EFD1C9
:1059C0004B469E60DF6004239C460433E2449C46C1
:1059D000059BE144E0449945D4D1079B0593B4E687
:1059E00000260027ECE732003B000020864902F049
:1059F000D3FA06000F00002C00D175E7069A0020AC
:105A0000814900F0ABFB02000B003000390002F0CE
:105A1000C3FA06000F0067E7069B002B12D1059B17
:105A200012AA013B9B00D558EB1507930DE7059B88
:105A300012A95A1E920012AB9B5810935B025B0A8C
:105A40008B504EE70022714B01F060FA00280ED116
:105A50000023079348E7534600260027C0C39A4611
:105A600008239C46E144DA4500D03AE659E6012392
:105A70009C4601330793059BE044002B00DDEEE6D6
:105A800032003B000020604902F086FA06000F0059
:105A90002AE743460B93069B12A8183B190006936E
:105AA0009300C3580092002B0FD156481300844630
:105AB00012A8634484469B006344043B5868013A3F
:105AC00018390028F9D000920691069A00204E4914
:105AD00000F044FB009B04000D00002B00DAB3E152
:105AE00012AA94469F00DB0067449C460A9A0593DD
:105AF000624493461600386802F0D8FD22002B005D
:105B000001F0D0FF424B306071600022200029007C
:105B100001F0C8FF083E74AB04000D00043FB3421F
:105B2000E9D100239A464EAB0293089B99464B4617
:105B300000260027002B21DB8020364B5D4698464F
:105B4000C005354900260027002408E008239C46AC
:105B50000835E044A24511DB4346186859682A68B5
:105B60006B6801F09FFF02000B003000390001F06C
:105B70005FFB013406000F00A145E7DA029A5346A5
:105B80009446DB0063441E605F6001239C46093B32
:105B9000E2449C4674ABE3449B45C8D1029B9946C2
:105BA000A89B022B00DD82E0002B37DC1DD1059B7A
:105BB00000254B441E000024326873682800210031
:105BC00001F036FB009B05000C00083E5A1E0092B7
:105BD000F2D2079B002B03D080231B069C46644413
:105BE0002A00230009990A604B6007200B9B18408C
:105BF0009F239B009D443CBC90469946A246AB46E1
:105C0000F0BDC046FFFFFF3F0000F03F0000E03F57
:105C10000000703E48AB0000FB21F93F059B0020CF
:105C20004B441E0000214CAF32687368083E01F0FF
:105C3000FFFABE42F8D1079B002B24D08023099A9B
:105C40001B06CB18106053600B0002004E984F9952
:105C500002F0A2F9009B002B0BDD012450AD0CCD0E
:105C600001F0E6FA009B0134A342F8DA079B002B0F
:105C700003D080231B069C4661440B000200099957
:105C80008A60CB60B1E702000B00099C2260636070
:105C90000B0002004E984F9902F07EF9009B002BFA
:105CA000DBDC0B00020009998A60CB609DE7A89BB2
:105CB000032B9AD1009B002B00DCE3E07E4A059B7E
:105CC00094464B441E685F68009B63449A46DB0021
:105CD0004B4498464CAB9B4643465C681B68180097
:105CE000210032003B000290039101F0A1FA040070
:105CF0000D0002000B000298039902F04DF93B00E1
:105D0000320001F095FA43469860D9601C605D60EE
:105D100008235B429C46E04426002F00C345DBD1AC
:105D2000009B012B00DCADE0059BC8464B441E6880
:105D30005F685346DB009B46D844434630005C68AE
:105D40001B683900009301941A00230001F070FAD7
:105D500004000D0002000B000098019902F01CF9EC
:105D60003B00320001F064FA43469860D9601C6041
:105D70005D6008235B429C46E04426002F00C1453D
:105D8000DBD15D460027002408354D4450AE2A681B
:105D90006B683800210001F04BFA083D07000C0049
:105DA000AE42F4D1079B002B71D0099A4E994B4615
:105DB0001160802109068C465B6849466344536044
:105DC0004B46DB688968634464449160D360176123
:105DD00054610AE7994643460B93069B30005A42AA
:105DE000390000F0BBF90022344B04000D0001F033
:105DF0008DF8002832D0324B00222000290001F01B
:105E000051FE02F01DFC4A460600970002F04EFCCF
:105E100000222A4B01F046FE02000B002000290060
:105E200002F0BAF802F00CFC12AAD0514A46069BC6
:105E30000132183300920693930012AAD65044E61A
:105E400001227FE500243AE5A89B022B14DC002BFD
:105E50000FDC00D0C9E600250024BAE64B4620003E
:105E600029009E0002F0ECFB12AB98514B460093C8
:105E70002BE600200021DEE64EAB9946A89B032BC3
:105E800000D0B2E6079B00270024002B8DD14E9A4C
:105E90004F9B09990A604B604B469A68DB680092F9
:105EA00001938A60CB603A0023000A614B619CE653
:105EB00076AB0A9335E4C046FFFFFF1F0000704138
:105EC0000000703EF0B54F464646C0B487B0009221
:105ED0000193464A4B00814688465B08934205DCA5
:105EE00002F0AEFB4146031E484666D04A46434692
:105EF0004846414601F0D6FD04000D0002000B00AB
:105F00004846414601F0CEFD394A3A4B06000F00A3
:105F10002000290001F0C6FD374A384B02F03CF85A
:105F200022002B0001F0BEFD354A364B01F080F90E
:105F300022002B0001F0B6FD334A344B02F02CF85E
:105F400022002B0001F0AEFD314B324A01F070F916
:105F50000E9B02900391002B34D0009801990022EF
:105F60002D4B01F09FFD029A039B04900591300098
:105F7000390001F097FD02000B000498059902F02A
:105F80000BF822002B0001F08DFD009A019B02F01E
:105F900003F8224A04000D00214B3000390001F0C3
:105FA00081FD02000B002000290001F041F90200F0
:105FB0000B004846414601F0EFFF07B00CBC90468D
:105FC0009946F0BD02000B002000290001F06AFD97
:105FD000124A134B01F0E0FF32003B0001F062FD7A
:105FE0004A46434601F024F9E7E7C046FFFF3F3E3B
:105FF0007CD5CF5A3AD9E53DEB9C2B8AE6E55A3E53
:106000007DFEB157E31DC73ED561C119A0012A3FEE
:106010001111813FA6F810110000E03F4955555578
:106020005555C53F49004B0819007047454AF8B51A
:10603000564692464B005B0D9A444D465F46444699
:106040005246F0B4894605000C000E000700132AE2
:1060500022DC002A47DB52463B4B134198460B009B
:1060600042461340034311D0384A394B01F0E0F85F
:106070000022002300F040FF002805D0002C41DB67
:106080004E46434600279E43380031003CBC9046B4
:106090009946A246AB46F8BD5246332A08DD802316
:1060A000DB009A45F2D102000B0001F0C1F8EDE7E8
:1060B000284A9446012263445242DA4093460242FF
:1060C000E4D0224A224B01F0B3F80022002300F072
:1060D00013FF0028D8D0002C1ADB5B464E469F43A6
:1060E00038003100D2E7194A194B01F0A1F800221B
:1060F000002300F001FF0028C6D0002C16DB00278B
:106100000026C1E7802352465B0313419944B7E759
:106110005346142B12D03423524601279B1A9F401A
:106120007F19AF429B415B429944D6E76400640803
:1061300025430027002DA7D0074EA5E7133B9C461B
:10614000E144CAE701FCFFFFFFFF0F009C750088D8
:106150003CE4377EEDFBFFFF0000F0BF4B0070B565
:106160005B0D14000A00002B1AD14B005B0803439F
:1061700015D00022224B01F095FC224B0A009C42D4
:1061800022DB4B005B0D363B1F4DE318AB4220DC9E
:10619000002B0DDD1D4C1B0522401A43110070BD64
:1061A0001B4DAB42F0D102000B0001F041F8F6E7C5
:1061B0001D00353518DA174B02009C420ADC0B0033
:1061C0001548164900F032F8134A144B01F06AFCE6
:1061D000E5E702000B001248124900F027F8104AC8
:1061E000104B01F05FFCDAE7084C363322401B0508
:1061F0001343190000220C4B01F054FCCFE7C046BA
:1062000000005043B03CFFFFFE070000FFFF0F807F
:10621000FF07000050C3000059F3F8C21F6EA5012C
:106220009C7500883CE4377E0000903C30B54A0005
:10623000DB0FDB0752081A43110030BD03210A4867
:1062400002680A430260094802680A43026008497A
:10625000084A094B9B1A03DD043BC858D050FBDCAD
:1062600000F0B4F9F9F786FF24050040540500401A
:106270001CAE00000000002040020020FEE7FEE708
:10628000FEE7FEE7FEE7FEE7014B18607047C046F9
:106290007C010020F7B50023202877D83C4B8000F4
:1062A000C258042A14D006D8022A0DD00ED80423CE
:1062B000012A14D069E0062A0ED00BD31A2A0DD079
:1062C00002231B2A0BD060E0082308E0102306E01D
:1062D000202304E0402302E0802300E001232D4A34
:1062E0001268082A04D9092A05D00A21022404E0E8
:1062F0000821002401E011000124A02501261C270B
:106300002548ED004651254D254E2D681B02AD0058
:106310003D400195234D2D6800958559AC46674653
:10632000214D3D401D4385518359C0259C46009B0E
:10633000AD021D40FF2367461B023B402B43019DDE
:106340001D43009B5F0160231F402B003B431C4308
:1063500001238451154C036063680F48002BFBD068
:106360000024124B01255C60A123DB00C35845606B
:10637000A025ED0044511BB2914207D002D98A1AE0
:10638000D34003E0521A934000E000231800FEBD02
:1063900018A9000080010020007000407801002052
:1063A0000405000074010020FF00FFFFFC700040A6
:1063B000F0B520286CD8374B8000C258364B1E6889
:1063C000002E2ED1C2243548A4000759344B032592
:1063D0003B40C0273F023B4303518023893C9B0045
:1063E000FF3C03512F4F03602F4B803CD859FF3C9B
:1063F000A043D8510437D859A8432043D85108376F
:10640000D8590C35A843083D2843D851A820C000CE
:106410001E508026C120760280001E501C601E4B3C
:106420001C6000231426214834005C4325580400D6
:106430006F1C0FD1142058432250A0200325C132D5
:10644000FF329200C0051550194A08001268082A48
:1064500003D10BE0AA4218D1ECE7082A02D9083A86
:10646000D14002E00820821A9140080014225343D0
:10647000E3189A680C495132FF329200586050502C
:10648000DA68C1239B00CA5002E00133032BCBD151
:10649000F0BDC04618A900008811002000E100E00E
:1064A000FF00FFFF04050000009000408401002071
:1064B0007C0100201E4BF0B5596C18001D4A0029C4
:1064C00014D0A025A12600230124ED05F600D15803
:1064D0004F1C06D0D7187F68002F02D027008F40AE
:1064E000AF5114333C2BF2D100234364131DA0257C
:1064F00040329446002001240F4EED05DA680F4922
:10650000920057180A495218526C002A0CD01A1FD0
:106510001268511C05D01968FF2902D02100914052
:10652000A9513A00FC32506414339C45E6D1F0BDC9
:10653000FC900040840100200C0500000090004009
:1065400000B5202816D80C4A83009B58032911D87F
:10655000A0220800C133FF33D2059B0000F014FBDA
:1065600002080406002104E00C2102E0042100E0FE
:106570000321D15000BDC04618A9000020280DD825
:10658000074B8000C058A0220123D2058340002978
:1065900001D1044901E0A121C90053507047C04610
:1065A00018A900000C05000003000020202B0AD8C9
:1065B000A222A021D200C9058858034A9B009B58FB
:1065C000D84001231840704718A900002D4B10B582
:1065D0001A78012A19D12C4A1268120715D12B4AB0
:1065E000E0241168F0220800104021420BD1284914
:1065F0000968114209D12749274A11608021274A99
:106600000902116001E03028F1D01A78012A0DD179
:106610001D490968090709D1F0201C490968014092
:10662000402903D11A490968014223D01B68DBB213
:10663000012B25D1144B1B681B0721D1134B1A6862
:10664000F0231A40A02A04D1114A12681A4203D03A
:1066500016E0D02A14D1F7E7114B1A68012A03D1AA
:10666000C022104B1A600BE00F4A1A601A68012A08
:10667000FCD1F5E7C1218020C900C0054250D5E713
:1066800010BDC046E00F00F0E40F00F0E80F00F08E
:10669000EC0F00F0DFFF07C004050040186C00405D
:1066A00000EC064014EC064075930000F7B50600B8
:1066B0000D000C008B180193019B671B9C4207D0B7
:1066C000336821781B683000984701340028F3D1E3
:1066D0003800FEBD70B505000C00081E07D002F0A2
:1066E0004FFD2B6802005B6821002800984770BDB1
:1066F00010B5FFF7EFFF10BD10B5402200210400D8
:1067000002F011F9002320002364636410BD3F23CD
:10671000026C10B5541C2340446C9C4201D081543F
:10672000036410BD0023036443647047436C026C30
:10673000934206D03F21C25C01330B4043641000FA
:1067400001E0012040427047036C406C181A00D5EC
:1067500040307047436C026C934201D0C05C01E052
:10676000012040427047036C406C5A1C3F23134089
:10677000181A42424241D0B270470120704710B50A
:1067800003681322DB69984710BD70470369054A07
:106790009950FC331A6A002AFCD0002201201A62A8
:1067A0007047C0461C050000030010B55C331A7822
:1067B0001F2313400122110099400D4B0424D96777
:1067C000C221036989005C505A60DA60A02200216E
:1067D000D20099500122074952425A5006491430BA
:1067E0005A500C395A5008315A50FFF79BFF10BDD0
:1067F00004E100E00C0500001405000010B51430A1
:10680000FFF7A2FF10BD10B51430FFF7A3FF10BDB6
:1068100010B51430FFF78AFF10BD0000030070B5FB
:106820005E331C780269604BD45003005D331C78E2
:106830005E4BD450030061331C785D4B012C0CD1AE
:1068400005005F352E78A225ED0056510500603514
:106850002E78A125ED00565100E00024D450962357
:10686000DB00994238D996231B01994237D99623E8
:106870005B01994236D996239B01994234D9E12391
:106880009B01994232D99623DB01994231D9E12308
:10689000DB0199422FD996231B0299422DD9E1237E
:1068A0001B0299422BD996235B02994229D9E123F5
:1068B0005B02994227D9E1239B02994225D93D4B9E
:1068C000994224D9E123DB02994223D9E1231B0316
:1068D000994221D8384B21E09E23DB021EE09D2304
:1068E0001B031BE0354B19E0354B17E0EC239B03F2
:1068F00014E0344B12E0344B10E0344B0EE0344BD8
:106900000CE0344B0AE0344B08E0344B06E08023C3
:10691000DB0403E0324B01E080235B0531490024B6
:1069200053500423243953501100FC31CC600C62C5
:10693000C1210134890014605C30946053500378A5
:106940001F202200D9B20840824080342648FF34FC
:106950005BB20251002B13DA0F230B40083B234C90
:106960009B089B001B1903242140A140FC348C4050
:10697000DD69A543C0248C4021002943D96111E081
:10698000194C9B089B001B1903242140A140C025E2
:10699000FC348C40AD005E59A643C0248C402100DD
:1069A00031435951026070BD0C0500001405000010
:1069B0006C05000090D0030000D0BE0E00B01300A4
:1069C0000050270000A04E0000F0750000509D0010
:1069D00000F0EB0000903A0100E0D70100B0AF03F7
:1069E00000705F072405000000E100E000ED00E01A
:1069F000F7B5009308AB1B7800250193FA23040038
:106A00009B0083600E4B45600833036014300F0019
:106A10001600FFF771FE23005C3327611E70009B98
:106A2000084A9B00995823005D331970019B200090
:106A30009B009A5823005E33DD701A70FEBDC0467D
:106A400088AB000018A90000036910B51A00FC32D9
:106A5000D2680400002A0AD0A322D2009958143028
:106A6000C9B2FFF754FE00222369FC33DA6010BD7F
:106A700010B50248FFF7E8FF10BDC0468C1100209A
:106A8000162307B5022200930249013B0248FFF793
:106A9000AFFF07BD002000408C11002070470000B0
:106AA00010B500F047F8FFF7F9FF012000F024F8D7
:106AB000FDF760FFFDF772FF024B002BFAD000E0FC
:106AC00000BFF7E700000000084A0949094B10B56C
:106AD0001B688858FA22190A1B06184392000023E3
:106AE00000F01EFA4904C00B084310BD0405000065
:106AF00000100140F011002070B5041E09D0FFF70E
:106B0000E3FF050000F014F8FFF7DEFF401B8442AE
:106B1000F8D870BD0022044B9A60044A1368013310
:106B2000DBB213607047C046FC100140F01100203A
:106B300070470000C421114A89005058104B03408F
:106B4000C020000203435350802391399B02FF3938
:106B5000535013608023A3220021DB05D2009950FB
:106B60000122A1209A60074BC0001950C1200231B8
:106B700080001950403019501A60704700E100E061
:106B8000FF00FFFF0010014002B4714649084900B0
:106B9000095C49008E4402BC7047C046002243088D
:106BA0008B4274D303098B425FD3030A8B4244D3D5
:106BB000030B8B4228D3030C8B420DD3FF22090217
:106BC00012BA030C8B4202D31212090265D0030BD6
:106BD0008B4219D300E0090AC30B8B4201D3CB03CC
:106BE000C01A5241830B8B4201D38B03C01A52410E
:106BF000430B8B4201D34B03C01A5241030B8B4210
:106C000001D30B03C01A5241C30A8B4201D3CB02FA
:106C1000C01A5241830A8B4201D38B02C01A5241DF
:106C2000430A8B4201D34B02C01A5241030A8B42E2
:106C300001D30B02C01A5241CDD2C3098B4201D3FA
:106C4000CB01C01A524183098B4201D38B01C01A78
:106C5000524143098B4201D34B01C01A52410309EF
:106C60008B4201D30B01C01A5241C3088B4201D39E
:106C7000CB00C01A524183088B4201D38B00C01A4B
:106C8000524143088B4201D34B00C01A5241411A72
:106C900000D20146524110467047FFE701B500207F
:106CA00000F0F0F802BDC0460029F7D076E7704743
:106CB00003460B437FD4002243088B4274D303095D
:106CC0008B425FD3030A8B4244D3030B8B4228D3FE
:106CD000030C8B420DD3FF22090212BA030C8B4224
:106CE00002D31212090265D0030B8B4219D300E0C4
:106CF000090AC30B8B4201D3CB03C01A5241830B49
:106D00008B4201D38B03C01A5241430B8B4201D3F8
:106D10004B03C01A5241030B8B4201D30B03C01A21
:106D20005241C30A8B4201D3CB02C01A5241830A9B
:106D30008B4201D38B02C01A5241430A8B4201D3CA
:106D40004B02C01A5241030A8B4201D30B02C01AF4
:106D50005241CDD2C3098B4201D3CB01C01A52415B
:106D600083098B4201D38B01C01A524143098B42E4
:106D700001D34B01C01A524103098B4201D30B01CD
:106D8000C01A5241C3088B4201D3CB00C01A5241F2
:106D900083088B4201D38B00C01A524143088B42B7
:106DA00001D34B00C01A5241411A00D20146524150
:106DB000104670475DE0CA0F00D04942031000D36F
:106DC0004042534000229C4603098B422DD3030AC4
:106DD0008B4212D3FC22890112BA030A8B420CD3D4
:106DE000890192118B4208D3890192118B4204D3FD
:106DF00089013AD0921100E08909C3098B4201D37D
:106E0000CB01C01A524183098B4201D38B01C01AB6
:106E1000524143098B4201D34B01C01A524103092D
:106E20008B4201D30B01C01A5241C3088B4201D3DC
:106E3000CB00C01A524183088B4201D38B00C01A89
:106E40005241D9D243088B4201D34B00C01A524160
:106E5000411A00D20146634652415B10104601D3ED
:106E60004042002B00D54942704763465B1000D377
:106E7000404201B5002000F005F802BD0029F8D01D
:106E800016E770477047C046D0400B1C1141203AAE
:106E900003D49C461341184363465242934018431F
:106EA0007047C0468446101C62468C46191C6346D7
:106EB00000E0C0461FB500F08BFD002801D4002182
:106EC000C8421FBD10B500F0DFFC4042013010BDCC
:106ED00010B500F07DFD002801DB002010BD012071
:106EE00010BDC04610B500F073FD002801DD002084
:106EF00010BD012010BDC04610B500F005FD0028F2
:106F000001DC002010BD012010BDC04610B500F00E
:106F1000FBFC002801DA002010BD012010BDC04696
:106F2000F0B54F464646C0B41604360C99463300B9
:106F300005042C0C070C150C63437E436F4365431B
:106F40001C0CAD1964199C46A64203D980235B0230
:106F5000984647446346250CEF191D044B464A43A7
:106F600043432D0C240464199918C91920000CBC42
:106F700090469946F0BDC046F0B557464E46454648
:106F80004300E0B446028846760A1F0EC40F002F65
:106F900047D0FF2F25D0002380259A469946F6003A
:106FA000ED042E437F3F434642465D02D20F5B0015
:106FB0006D0A1B0E904640D0FF2B39D08022002056
:106FC000ED00D20415437F3BFB1842465746591C3F
:106FD00062408C4607430F2F5CD86F49BF00C959E8
:106FE0008F46002E45D108239A46063B9946DAE79C
:106FF000424602282DD0032800D1C3E0012800D04A
:10700000A2E0002500260240D4B27602ED05760A01
:107010002E43E407264330001CBC90469946A24606
:10702000F0BD002E1AD104239A46033B9946BAE7D5
:107030002A00511E8A41901CC6E70120002DC3D0B2
:10704000280001F0C9FB431F76309D4043420020D9
:10705000BAE70124FF2514400026D6E7300001F0EE
:10706000BBFB431F9E400023763047429A46994619
:1070700099E70C239A46093B994694E78026002419
:10708000F603FF25C1E735004846B2E73500220088
:107090004846AEE72904090C0800370C3604360CC4
:1070A0002C0C7943704367437443060C64183619FB
:1070B000B14203D980214902884647440004000CAC
:1070C000310409188D01681E8541890E2943350C4C
:1070D000ED19AD010D43290104D5012369081D40B7
:1070E00063460D4319007F31002925DD680704D070
:1070F0000F202840042800D00435280103D5274953
:1071000080330D401900FE29A3DC0124AD016E0A75
:107110001440CDB279E78020C003064207D0054273
:1071200005D128434602760A4446FF256DE706430B
:107130007602760AFF2568E70124611A1B2905DD1E
:1071400014400025002660E76346CBE72E0020238D
:10715000CE40591A8D406B1E9D412E43730704D0BB
:107160000F233340042B00D00436730104D50124CF
:1071700001251440002648E70124B601760A144090
:10718000002542E780260124F6032E437602760A84
:107190001440FF2539E7C046B8AB0000FFFFFFF7FA
:1071A00070B5002830D0C317C5185D40C40F280043
:1071B00001F012FB9E231B1A962B0DDC9622D21A8D
:1071C00095406A02520AD8B25202C005520AE40738
:1071D00002432243100070BD992B19DC9922D21A68
:1071E0009540124A2A40690704D00F210D40042D12
:1071F00000D00432510103D50C4B1A409F231B1AB7
:107200009201520AD8B2DFE7002400200022DBE717
:1072100005222E00121AB921D6402A00C91A8A4026
:10722000551EAA4135001543DBE7C046FFFFFFFBB3
:10723000F8B556465F464D464446F0B40F00FD0F84
:10724000AA4609037C002E005F00450F490A7F0D06
:107250002943C5001803BC46400A570F640DDB0FD5
:107260003843D2009A4500D1AAE06646A61B002EFC
:1072700000DCFFE06346002B39D10300134300D04C
:10728000D9E06B0709D00F232B40042B05D02B1D11
:10729000AB42AD416D4249191D000B0200D482E0A2
:1072A000CA4B01349C4200D1FEE00A005646C84B4E
:1072B000ED081A405007640552020543120B640D95
:1072C000002112030B0D1B056405120B1A43630802
:1072D000C04CF60714401C43640064083443280083
:1072E00021003CBC90469946A246AB46F8BDB74B40
:1072F0009C42C6D080231B041843382E00DDEBE0EF
:107300001F2E00DD1EE120239B1B9C4603006746C9
:10731000BB40984613004746F3403B436746BA409C
:10732000571EBA4113430200F240EB1A9D42B64188
:107330001D008A1A7642911B0B0231D54A02560A69
:10734000002E00D1B4E0300001F046FA0300083B03
:107350001F2B00DDB5E020222900D21AD1409E402B
:107360000A009D4032439C4200DDB1E01C1B631CBF
:107370001F2B00DDD5E0202114002800C91A8C4005
:10738000D8408D400443DA40681E854111002543F2
:10739000002476E74146314300D134E231004546CE
:1073A0006B0700D06FE756464807ED08C90805434C
:1073B000864B9C4235D00A036405120B640D7FE7AF
:1073C0006346E31A9B46002B00DC8BE06746002FE8
:1073D0003CD07E4FBC4200D153E780273F04384366
:1073E0005B46382B00DCF7E00243501E8241002050
:1073F000D2B253194218AB4289411D004942891843
:107400000B02CDD5714B01349C4200D13DE10120EE
:107410006F4A6B080A4028401843D50705435108B6
:107420002FE72B000B4300D1CBE180231B030B4341
:107430001A03120B44E7013E002E6DD1AE1AB5427D
:107440009B41091A5B42C91A350075E707001743CB
:1074500000D116E701235B429C46E3445B46002BC8
:1074600000D0E0E0AA18AA429B4109185B425918D3
:107470001500C5E7002E75D1661C7605760D012E28
:1074800000DCF3E0AE1AB0464545BF410E1A7F421C
:10749000F61B370200D48FE0551BAA42B641411AB1
:1074A00076428E1B9A464BE756460022002507E798
:1074B000280001F091F920300300083B1F2B00DC6D
:1074C00049E72A002838824000259C4200DC4DE72D
:1074D0003F49E41A1140D4E60243501E8241D3B220
:1074E000002222E7002B00D0F3E0631C9C465B05E2
:1074F0005B0D012B00DC9FE0344B9C4500D1C3E0C9
:10750000AA180918AA42804140424118CD075208E2
:10751000154349086446B4E62C4B9C4200D0ECE687
:10752000AFE611001F3CE1400C00202B00D17FE0B2
:107530004021CB1A9A4015436A1E954100212543EC
:1075400000242DE733000700203BDF403B00202EC6
:1075500070D04027BE1BB0400243501E82411343EF
:107560000022E2E6002C4FD0184CA44500D1ABE03D
:107570008024240476422143382E00DDDFE01F2ED4
:1075800000DD43E12027BC1BA1460C004F46BC4058
:10759000A0462C004746F4403C434F46BD406F1E7A
:1075A000BD41F1402C43151BAA429241411A52425F
:1075B000891A64469A46BFE641464546314300D0A3
:1075C000BEE6002600240025F2E6C046FF070000C4
:1075D000FFFF7FFFFFFF0F801F2B59DC2027FF1AC3
:1075E000BC46070063469F405B46B9461700DF4034
:1075F000B8464F4643461F4363469A40531E9A413E
:107600005B463A43D840F4E60C002C435CD0F6438A
:10761000002E55D1551BAA42A441411A6442091BB0
:107620009A46644688E6964FBC4200D0D8E628E6E3
:10763000002280E700208FE70B002B43002C00D0B6
:10764000C2E0002B00D101E10300134300D118E692
:10765000AB18AB42B6410918764271180A0200D441
:1076600009E1884A1D00114064460AE6002C5BD1FE
:107670000E002E4300D08AE00100114300D1C2E089
:10768000010015009A46FCE56446002100258FE6BE
:1076900020235B429C46DC4463460700DF405B4698
:1076A000BC46202B00D1ACE040235F46DB1B98405A
:1076B0000243501E8241634613431A00002098E69D
:1076C0006F4CA44500D057E70100150064469A4668
:1076D000D7E5002C39D10C002C436ED0DB43002BB6
:1076E0001AD0674CA44568D0382B00DDA4E01F2BCE
:1076F00000DDAEE020240F00E41AA740B9462F00B9
:10770000DF40B846A3464F46444627435C46A54063
:107710006C1EA541D9403D43AD1895429B410918C7
:107720005B42591864466BE60C002C4315D10100EE
:1077300011437BD0010015009A46514CA1E50D4341
:10774000691E8D410021ECB22DE74D4CA44534D08B
:10775000802424045B422143C6E7040014434ED036
:10776000ED084C072C438025C9082D03294208D079
:10777000C6082E4205D1D208410711430C009A4693
:107780003100620FC900E50011433D4C79E5060068
:10779000164300D175E5AE1AB0464545BF410E1AF5
:1077A0007F42F61B370200D4F4E5551BAA42B641CE
:1077B000411A7642891B9A4663E50100150064462A
:1077C0005FE5002200257BE5002B3BD0030013433F
:1077D00015D0ED084B072B438025C9082D032942FE
:1077E00007D0C4082C4204D141070B002100D20865
:1077F0001343C9005A0F1143DD00214C41E5204CD1
:107800003FE5002054E700260025D1E534000F00B5
:10781000203CE7403C00202E2BD04027BE1BB1402F
:107820000D43691E8D4100212C43BCE680210026BA
:107830000903134C0025BBE50D43691E8D41002152
:10784000EDB269E7010015000D4C1AE501001500C5
:1078500017E51C000F00203CE7403C00202B0CD01B
:107860004027FB1A99400D43691E8D410021254395
:1078700052E70021D4E71D0092E50021F3E7C0465E
:10788000FF070000FFFF7FFFF0B55F4656464D46FD
:107890004446F0B41F035C00DB0F9A46194B0E03FD
:1078A0004D00C90F8046360B6D0D8B4691463F0B40
:1078B000640D9D4219D0134B9C421BD00123A5425D
:1078C00006D018003CBC90469946A246AB46F0BD97
:1078D000BE42F6D1C845F4D1D34510D0002DF0D129
:1078E000304303005A1E9341EBE73100012301436B
:1078F000E7D1E0E73A430123002AE2D1DEE70023A3
:10790000DFE7C046FF070000F0B55F464446564635
:107910004D46F0B41F033C0B2C4F0E034D00A34605
:107920005C008446360B6D0DC90F9046640DDB0F6D
:10793000BD422BD0254FBC422ED0002D0ED130435E
:107940000700814678427841002C17D15F463A43C0
:1079500014D14B460020002B0AD006E0002C02D1A7
:107960005846024301D099421AD001234842184395
:107970003CBC90469946A246AB46F0BD0028F2D0EA
:1079800058425841012240421043F1E73700074373
:10799000D0D002204042EBE75F461743CDD0F8E756
:1079A000A542E2DC05DB5E45DFD808D000205E455D
:1079B000DED248424841012340421843D8E7C4453B
:1079C000D3D80020C445F4D3D2E7C046FF07000057
:1079D000F0B55F464D4644465646F0B41C03240BB2
:1079E000A4462F4C0F034D005E00C90F80463F0B8D
:1079F0006D0D8B469146760DDB0FA54220D0284CAD
:107A0000A64222D0002D12D1384344424441002ED8
:107A100020D0002C0DD05C42634101245B421C430A
:107A200020003CBC90469946A246AB46F0BD002ED5
:107A300017D05B4519D05B465C4201231C43EFE73E
:107A4000390002240143EBD1D9E7614602241143F6
:107A5000E6D1D7E761460A43DBD100240028DFD016
:107A6000E9E761460A43E4D1E5E7B54203DD0122D7
:107A70005C421443D4E7B542CDDB6745DBD809D07F
:107A800000246745CCD259464C4261410124494209
:107A90000C43C5E7C845CED80024C845F3D3BFE79B
:107AA000FF070000F0B55F4656464D464446F0B429
:107AB0000D0399464E002B0B87B007009246804677
:107AC0009B46760DCC0F002E69D06D4B9E4235D073
:107AD0005B468022DD001204430F13432B439B4679
:107AE000C3009846674B00279C46002366440193D9
:107AF0004A4615035000D20F53462D0B400D9146B8
:107B000000D176E05E4A90426CD080225B0F120476
:107B100013435C4AED0094461D4353460022DB00AC
:107B2000604449463618701C6140029017430F2F7D
:107B300000D9AFE05448BF00C759BF465B461F435A
:107B400000D088E000239B46984602330827019323
:107B5000CEE74946022A6AD0032A00D109E2012A67
:107B600000D0BBE111400022002300259046CCB29A
:107B700000212D030A0D12052D0B1543434A1B0549
:107B800015401D436D00E4076D082543404629005C
:107B900007B03CBC90469946A246AB46F0BD0343B5
:107BA00052D05B46002B00D18AE1584600F014FE0B
:107BB00003000B3B1C2B00DD7BE11D22D31A3A0096
:107BC00001005D46DA4008398D4013008F402B4399
:107BD0009B46B8462E4B00279C46002360444642F5
:107BE000019385E752462A432CD100250023022227
:107BF00097E752462A4321D0002D00D154E12800B6
:107C000000F0EAFD03000B3B1C2B00DD46E11D21CB
:107C1000CB1A51460200D9405346083A954093404A
:107C20000D431B4A944660444042002279E70124F8
:107C300000220C40124B0025904699E700250023B6
:107C400001226EE703226CE700239B46984601332E
:107C5000042701934CE703230C27019348E70023F3
:107C60008025984600242D03054B81E75D46434659
:107C7000019A6FE75D4643462100019A6AE7C046D4
:107C8000FF07000001FCFFFFF8AB0000FFFF0F80C3
:107C9000F30300004246120C91461A0C94464246E9
:107CA00017044A461B041B0C5A43604690464A463A
:107CB00042431000039262461C003F0C7A437C430F
:107CC00042440192220C9246019A5244904506D9B0
:107CD0008246802040028046C24450460390100CE9
:107CE000049048462404240C1204121905922A0C0C
:107CF0002D042D0C68432C00824648467C4350439B
:107D00008146200C8046574357444744BA4503D91F
:107D1000802040028046C144380C3F04B8464844A5
:107D20002404240C01900498A04440440490584634
:107D3000000C814658460404200C82460700484641
:107D40005F434C4643436046604364468346504627
:107D50004443380C8446E4186444A34203D9802386
:107D60005B029C46E34448463F04230C3F0C24043A
:107D7000E419574668436F4384464D465046554381
:107D80004243380C814662444A445B44944503D9DB
:107D9000802040028446654403983F04834604984B
:107DA0003F0C8446E344C345804140428246100470
:107DB00084460198674484466744A344BC46A3456F
:107DC000A4419946D44464428742BF41D44580418E
:107DD000E144A04699459B417F424042C844074345
:107DE000120CBA18A045A4415F423B0064422343F1
:107DF000D71843467D19DB0D6D021D435B465A02C1
:107E0000059B1A43531E9A415B46DB0D1A434346BA
:107E10005B021343EA0107D501225C0813402343A8
:107E2000EA07029E13436D08574AB218002A4BDD39
:107E3000580709D00F201840042805D0181D984273
:107E40009B415B42ED180300E80104D54F4A154001
:107E50008022D200B2184E48824200DDE7E60124BB
:107E6000DB08680718436D02530580462D0B5B0D38
:107E70000C407DE6802259461203114208D015427B
:107E800006D115432D0398462D0B4C46414B6FE60A
:107E90005D4615432D032D0B3E4B69E60300554609
:107EA000283B9D400023BCE6504600F095FC203066
:107EB000A8E60300283B9F400023BB46984689E67E
:107EC00000F08AFC203073E60124A61A382E07DD64
:107ED00000220C4000230025904649E6029EA3E7BD
:107EE0001F2E20DC20222C001800921BF040944012
:107EF00093400443581E83411C43F540630709D057
:107F00000F232340042B05D023001C1D9C429241CB
:107F10005242AD182B021FD5012400220C40012330
:107F20000025904624E61F202C004042821AD440AF
:107F3000202E1CD04022961BB5402B43581E834157
:107F40000720234318400025002809D00F220025D0
:107F50001A401C00042AD8D1230068076D022D0B9B
:107F60000124DB08034398460C40002300E600256B
:107F7000E3E780220124120315432D0398462D0BBD
:107F80000C40044BF4E5C046FF030000FFFFFFFE7A
:107F9000FE070000FF070000F0B557464E46454675
:107FA000E0B40E001100F20F9246C500420F180314
:107FB00037037400400A4E0F7F0A3043CF4E1743F9
:107FC0005A00640D520DDB0FC900B24200D1E5E04A
:107FD00001267340A61AB446534500D1AFE0002EE7
:107FE00000DC0DE1002A3AD103000B4300D0E4E0AD
:107FF0006B0709D00F232B40042B05D02B1DAB4260
:10800000AD416D427F191D003B0200D488E0BB4B9F
:1080100001349C4200D110E13A00B94B51461A405C
:1080200001235007ED08520264050543120B640D4D
:108030000B400021280012030D0D120B64052D05C5
:1080400015436208AF4CDB072C40144364006408FE
:108050001C4321001CBC90469946A246F0BDA74B8C
:108060009C42C5D080231B0418436346382B00DD97
:10807000FDE01F2B00DD30E1624620239B1A020049
:108080009A40664690460A009940F24046464B1E8A
:1080900099413243114363460200DA40691A8D4226
:1080A0009B410D00BA1A5B42D71A3B0235D57A02C2
:1080B000530A98464346002B00D1C4E0404600F0E6
:1080C0008BFB0300083B1F2B00DDC5E020222900AD
:1080D000D21A4746D1409F400A009D403A439C42F5
:1080E00000DDC0E01C1B631C1F2B00DDE4E0202131
:1080F00014002800C91AD8408C408D400443DA404F
:10810000681E854117002543002471E742466346F7
:108110001A4300D14CE2674645466B0700D069E739
:10812000012351467807ED08FA080B4005437349CF
:108130008C4238D012036405120B640D79E7002ECF
:1081400000DC9AE0002A47D06C4A944200D14FE705
:108150008022120410436246382A00DC08E1014301
:10816000481E81410022C9B24919D219A942BF4112
:108170000D007F42BF183A0200D442E15F4A013449
:10818000944200D14EE101205D4A69083A402840FE
:108190000843D507054357089A4629E706000E43CA
:1081A00000D017E714E72900114300D1F9E180213D
:1081B00009030A431203120B3BE701235B42984673
:1081C000C4446346002B72D1691A8D429B413F1A09
:1081D0005B42FF1A0D0068E702000A4300D107E77F
:1081E000012252429046C4446246002A00D0E6E092
:1081F0006918A942B6413F187642F7190D00BAE74F
:10820000002E00D080E0621C5205520D012A00DCD5
:10821000F9E06A1A91464D45B6413A1A7642921BE8
:108220009046120200D499E04D1BA9428941C71B18
:1082300049427A1A90469A463CE752460123002565
:1082400013400022F5E6280000F0C6FA20300300B3
:10825000083B1F2B00DC39E72A0028388240002524
:108260009C4200DC3EE7264FE41A1740C0E601437B
:10827000481E81410022C9B210E7002E00D0F1E073
:10828000621C94465205520D012A00DCA0E01B4AF4
:10829000944500D1C5E06918A94292413F18524265
:1082A000D2194908D5070D4357086446A0E6134B79
:1082B0009C4200D0D9E69BE611001F3CE1400C0037
:1082C000202B00D180E04021CB1A9A4015436A1E32
:1082D00095410027254300241FE763460200203B09
:1082E000DA406346202B71D0402366469B1B9840A2
:1082F0000143481E814111430022CFE6FF070000E1
:10830000FFFF7FFFFFFF0F80002C48D0CA4CA24226
:1083100000D1A2E07442A1468024240427434C46A5
:10832000382C00DDDBE01F2C00DD44E14E4620242C
:10833000A41B3E00A640A246B0464C462E00E64096
:10834000B4464646644626435446A5406C1EA541A5
:1083500034002C434D46EF400D1B28E04A4643466F
:108360004D461A4300D0A5E6002300240025DEE692
:108370001F2A5ADC66462022921B06009640914630
:10838000B04662460E00D640424616434A469140E9
:108390004A1E9141020060463143C240E4E63C007F
:1083A0002C435AD0F443A146002C52D14D1BA94274
:1083B0008941C71B49427F1A14009A4675E69E4AB6
:1083C000944200D0C7E613E600227FE700208FE743
:1083D000002C00D0C8E03B002B4300D10FE103008C
:1083E0000B4300D104E66918A9429B413F185B4248
:1083F000DF193B0200D41AE1904B0D001F40644688
:10840000F6E59A4689E63A002A43002C5CD1002A18
:1084100075D102000A4300D1CAE007000D009A4658
:10842000E6E564460022002581E662460600203A21
:10843000D6406246B046202A00D1B7E040226646C8
:10844000921B904001434246481E81411143002245
:108450008AE6794CA24200D061E707000D001400C3
:108460009A46C5E5002C41D13C002C4378D0F4431A
:10847000A146002C20D0704CA24271D04C46382C22
:1084800000DDB2E01F2C00DDBCE02026341BA2463C
:108490003C005646B4404E46A0462C00F440A4464C
:1084A000444666463443A4465446A54064466E1E80
:1084B000B54125434C46E7406D188D4289413F1830
:1084C0004942CF19140056E6002A2FD102000A4370
:1084D00000D184E007000D009A46574C88E53D43E3
:1084E0006F1EBD41ECB200270D1B60E7524CA2424B
:1084F00036D0744280263604A1463743BEE70200D8
:108500000A4300D174E56A1A90464545B6413A1AC5
:108510007642921B9446120200D4F7E54D1BA94205
:108520008941C71B49427F1A9A4661E502000A4306
:108530003AD0ED087C072C438025FA082D032A4207
:1085400008D0C7082F4205D145072C003A009A46AB
:10855000C9080C43670FD200E5001743364C47E5C6
:1085600007000D00140043E53A002A4343D00200FF
:108570000A4319D0ED087C072C438025FA082D0307
:108580002A4207D0C6082E4204D147073C003200D9
:10859000C9080C43D700620FE50017439A46264CE2
:1085A00026E50022002544E5234C21E5002049E78B
:1085B00000230025BBE54C463E00203CE6404C46EF
:1085C000B446202C31D040244E46A61BB7403D4334
:1085D0006C1EA54164462C4300270D1BE7E6802254
:1085E00000231203144C0025A1E53D436F1EBD413D
:1085F0000027EDB260E707000D000F4CF8E407001C
:108600000D00F5E44E463C00203EF440A0464C46AA
:10861000202C0ED040244E46A41BA7403D436F1E85
:10862000BD4144460027254346E70027CFE70D001C
:1086300073E50027F2E7C046FF070000FFFF7FFF5A
:108640000B0330B5134D1A0B4B005B0DC90F002403
:10865000AB4211DD104CA34210DC802464032243A2
:108660000E4CE41A1F2C0CDD0D48C31ADA4013001F
:108670005C42002900D11C00200030BD094BCC1801
:10868000FAE7E040084CA44663449A4013000343D1
:10869000EEE7C046FE0300001D04000033040000A6
:1086A00013040000FFFFFF7FEDFBFFFF70B5002804
:1086B00030D0C317C4185C40C50F200000F08CF800
:1086C000174B184A1B1AD21A1F2A18DD164AD21A3B
:1086D0009440002224035B05240B5B0D0021100055
:1086E00024030A0D1205240B1443104A1B051440E1
:1086F0001C436400ED0764082C43210070BD210079
:1087000091400A000B21081AC4405B052403240B86
:108710005B0DE3E70025002300240022DEE7C046CE
:108720001E0400003304000013040000FFFF0F804C
:108730004200120E511C4302C9B270B55D0AC40F4B
:10874000012915DDE02189008C466D071B0B624471
:10875000002128000D0D2D052B431C4D52052B40EB
:10876000520813435B00E4075B082343190070BD04
:10877000002A15D1002D1FD0280000F02DF80A285E
:108780001DDC0B232A001B1ADA40130002001532ED
:1087900095400F4A1B03121A52051B0B520DD7E7C7
:1087A000002D06D080221B0B120313436D07094ACC
:1087B000CEE7084A0023CBE700220023C8E70300E6
:1087C0000B3B9D402B000025E3E7C046FFFF0F80D9
:1087D00089030000FF0700001C2101231B049842AD
:1087E00001D3000C10391B0A984201D3000A083942
:1087F0001B09984201D30009043902A2105C4018F9
:108800007047C0460403020201010101000000009C
:10881000000000007FB51D000A4B06001B68D868E9
:10882000002A02D1084C230001E01300074C0293F8
:10883000009133002A000649019400F021F800F06D
:1088400023FEC0462002002009A2000038AC000030
:1088500045AC0000084B10B50400002B02D00021ED
:1088600000E000BF054B1868836A002B00D09847D2
:10887000200001F0F3FAC0460000000078AC0000D0
:108880000EB403B5010003AB044804CB00680193A8
:1088900000F016F902B008BC03B01847200200200F
:1088A0000E4B70B500251E000D4CE41AA410A54215
:1088B00004D0AB00F35898470135F8E701F0D0FA3F
:1088C000084B00251E00084CE41AA410A54204D051
:1088D000AB00F35898470135F8E770BD2802002037
:1088E00028020020280200203802002010B5034B87
:1088F0000100186800F066F810BDC0462002002094
:1089000010B5034B0100186800F016F810BDC04602
:1089100020020020002310B59A4203D0CC5CC4543E
:108920000133F9E710BD03008218934202D0197099
:108930000133FAE77047000030B500293ED0043912
:108940000B68002B00DAC9181D4A13681400002BAD
:1089500002D14B60116031E08B420DD90A68881852
:10896000834203D118685B6882180A604B602160FB
:1089700024E08A4203D813005A68002AF9D11D68FE
:108980005C198C420BD10968691858181960824229
:1089900014D110685268411819605A600EE08C4278
:1089A00002D90C23036009E008680C18A24203D125
:1089B00014685268201808604A60596030BDC0468B
:1089C000F8110020032370B5CD1C9D430835060027
:1089D0000C2D01D20C2505E0002D03DA0C2300201C
:1089E000336040E0A942F9D81F4B1C681A002100EF
:1089F000002913D00B685B1B0DD40B2B02D90B6025
:108A0000CC181EE08C4202D1636813601AE04B68F8
:108A100063600C0016E00C004968E9E7134C23681A
:108A2000002B03D1300000F033FB20602900300020
:108A300000F02EFB431CD1D00323C41C9C43A04256
:108A40000AD12560200007220B30231D9043C31A52
:108A500009D05A42E25006E0211A300000F018FB1B
:108A6000431CEED1BAE770BDF8110020F4110020CC
:108A7000936810B5013B9360002B05DA9469A3421B
:108A800008DBCBB20A2B05D01368581C1060197094
:108A9000C8B201E000F02CFC10BDF8B506000F00D4
:108AA0001400D518AC4208D021783A003000FFF706
:108AB000DFFF0134431CF5D100E00020F8BD0000C9
:108AC000F0B59FB006000F0002920593002804D075
:108AD0008369002B01D100F0D3FD7F4B9F4201D170
:108AE000776808E07D4B9F4201D1B76803E07C4B7B
:108AF0009F4200D1F768BB891B070AD53B69002B51
:108B000007D0002306AD6B6120336B761033AB7654
:108B10003DE03900300000F043FC0028F1D0012096
:108B20004042D6E0059A111D12680591002A00DA2C
:108B30007FE00992013423782E2B00D18DE021783B
:108B40000322684800F082FE002807D0654B2A689F
:108B5000C01A4023834013432B6001342178631CE7
:108B6000062261480293297600F070FE002800D1A9
:108B70009DE05E4B002B00D090E00722059B073361
:108B80009343083305936B69039A9B186B61029CAE
:108B90002378002B04D1029BE31A049312D003E044
:108BA000252BF8D00134F3E7049B029A39003000FA
:108BB000FFF773FF431C00D186E06A69049B94466B
:108BC00063446B612378002B7ED001220023524244
:108BD0006A6002A95432521801342B60EB60AB601A
:108BE0001370AB6521780522414800F02FFE002864
:108BF00008D03F4B2A68C01A0123834013432B60DF
:108C00000134EFE72B68DA0604D55322202102A8AD
:108C1000121811701A0704D553222B2102A812181A
:108C2000117022782A2A00D17CE7099B00200A21B2
:108C300005E05242EA60022213432B607AE7227871
:108C4000303A092A04D84B4301349B180120F6E737
:108C5000002800D16FE709936DE763782A2B0AD1CA
:108C6000059B02341A1D1B680592002B01DA0123B3
:108C70005B42079363E700230A201A0001346B600C
:108C800021783039092904D842430134521801238C
:108C9000F6E7002B00D152E7079250E705AB0093AF
:108CA0003A00144B2900300000E000BF07E005AB9C
:108CB00000933A000F4B2900300000F08BF803902E
:108CC000039B013300D05EE7BB895B0600D526E736
:108CD0000B981FB0F0BDC046B0AD0000D0AD000095
:108CE000F0AD000082AC000086AC00000000000087
:108CF0007CAC00009B8A0000F7B5170001938A68DE
:108D00000B6900900C00934200DA130022003B60D4
:108D100043321278002A01D001333B6023689B065E
:108D200002D53B6802333B60062523681D401ED0F8
:108D3000230043331B785A1E9341226892061CD5A8
:108D40003020E1184331087021005A1C4531097860
:108D5000A2184332023311700FE0220001231932AE
:108D600001990098089EB047431C0ED00135E36876
:108D70003A689B1A9D42F0DBDAE722000199433200
:108D80000098089DA847431C02D10120404220E0E2
:108D900006232068E1683A6803400025042B03D1CC
:108DA0008D1AEB43DB171D40A3682269934201DD56
:108DB0009B1AED180027BD420AD0220001231A3267
:108DC00001990098089EB047431CDED00137F2E7B6
:108DD0000020FEBDF0B58BB006920A004332079327
:108DE000059004920A7E0C00109B6E2A00D1ABE025
:108DF00011D8632A22D009D8002A00D1B5E0582A18
:108E000000D0C5E045310A70814A4FE0642A1DD088
:108E1000692A1BD0BCE0732A00D1AAE009D86F2AC6
:108E200029D0702A00D0B3E0202209680A432260CA
:108E300037E0752A1FD0782A33D0A9E00E001A68CF
:108E40004236111D196013683370A4E021681A6856
:108E5000080606D4490604D5111D19600023D55E05
:108E600002E0111D19601568002D3BDA2D23049ACC
:108E70006D42137036E021681A68080606D4490668
:108E800004D51568111D1960ADB202E0111D1960FD
:108E900015685F4B227E039308276F2A1DD00A278F
:108EA0001BE022007821453211705A4A196803925A
:108EB000081D226818600D68100602D4500600D5FF
:108EC000ADB2D30702D520231A4322601027002D0C
:108ED00003D1202322689A432260230000224333D7
:108EE0001A7002E00A274A4B03936368A360002BC1
:108EF00009DB0422216891432160002D05D1049EE5
:108F0000002B11D07BE0002D79D0049E2800390081
:108F1000FDF7CAFE039B013E5B5C280033703900FD
:108F2000FDF73CFE051EF1D1082F09D12368DB07B0
:108F300006D563682269934202DC3023013E337018
:108F4000049B9B1B23612BE009681A68080607D461
:108F5000490605D5111D19601368A28A1A8004E01C
:108F6000111D1960136862691A600023049E236151
:108F700016E01A68111D1960166800216268300039
:108F800000F064FC002801D0801B6060636803E08F
:108F9000260042363270012323610023049A1370A5
:108FA000079B09AA00932100069B0598FFF7A4FEE2
:108FB000431C02D10120404227E023693200069978
:108FC0000598079DA847431CF4D0236800259B07FC
:108FD0000FD4099BE068984217DA180015E02200C8
:108FE0000123193206990598079EB047431CE1D02A
:108FF0000135E368099A9B1A9D42F0DBE9E72600F8
:10900000039B42361B7833708EE70BB0F0BDC04631
:109010008DAC00009EAC0000154B10B51C68A36B16
:10902000002B15D11820FFF761FC124BA0630380C1
:10903000114B01224380114B8380114BC380114B94
:109040000381052343810633838100230261436149
:10905000A46B0D4A206961690C4BFDF761FF012289
:10906000002380185941206161614800400810BD0B
:10907000200200200E330000CDABFFFF34120000B1
:109080006DE6FFFFECDEFFFF2D7F954C2DF4515870
:10909000002370B5064C05000800236000F0C8FEF0
:1090A000431C03D12368002B00D02B6070BDC04649
:1090B000EC2400200CB430B5164B9DB00C1E1D687E
:1090C00004DA8B2301202B6040421DE0822302A999
:1090D0009B008B810023029008619C4200D0631E9C
:1090E0008B604B6101235B42CB81209A21AB28002E
:1090F000019300F053FC431C01DA8B232B60002CFE
:1091000002D00023029A13701DB030BC08BC02B01C
:109110001847C046200200200EB410B59DB002A929
:10912000029008610B488224886048610120404217
:109130001FABC881084804CBA400006801938C8150
:1091400000F02CFC0023029A13701DB010BC08BC68
:1091500003B01847FFFFFF7F2002002002780B7842
:10916000002A03D0013001319A42F7D0D01A70475B
:10917000031C0A7801311A700133002AF9D17047B3
:109180000023C25C0133002AFBD1581E7047030044
:1091900030B5002A0DD00C7801335D1E013A2C70D9
:1091A0000131002CF5D19A189A4202D01C7001337B
:1091B000FAE730BDF0B51E00454B87B01B68019241
:1091C000029308220B00059003911C7802995D1C04
:1091D00009194878104001D02B00F6E72D2C04D156
:1091E0009D1C5C780123009304E000902B2C01D19E
:1091F0005C789D1C002E02D0102E0AD162E0302C2B
:109200005ED120222B789343582B54D110266C78B2
:109210000235009F31007B1E9F412E4BFF18380006
:10922000FDF742FD380004913100FDF7B7FC002343
:109230000322070094461800029A1219517804225A
:10924000114201D0303C07E06246114017D037226E
:10925000012900D02032A41AA64210DD5A1C0BD0DE
:10926000B84207D802D1049B9C4203DC704301231F
:10927000201801E001235B422C780135DCE75A1C01
:109280000BD10098059A431E9841124BC018222317
:109290001360019B002B0AD117E0009A002A00D02E
:1092A0004042019A002A10D0039A002B00D06A1E77
:1092B000019B1A6009E03024002EAAD10826A8E7F5
:1092C0000A26A6E7302C9CD0A3E707B0F0BDC04625
:1092D00024020020FFFFFF7F10B513000A000100E9
:1092E00002480068FFF766FF10BDC046200200205C
:1092F000F8B505000F001400002804D08369002B86
:1093000001D100F0BDF9234B9C4201D16C6808E00B
:10931000214B9C4201D1AC6803E0204B9C4200D120
:10932000EC68A369A360A3891B070AD52369002BF6
:1093300007D023682269FEB2981A636998420FDB4E
:1093400008E02100280000F02BF80028F1D00120CF
:1093500040421DE02100280000F024F90028F6D149
:10936000A3680130013BA36023685A1C22601F7070
:109370006369984205D0A3893000DB0708D50A2E1F
:1093800006D12100280000F00DF90028DFD13000BF
:10939000F8BDC046B0AD0000D0AD0000F0AD00009B
:1093A000354B70B51D6806000C00002D05D0AB696B
:1093B000002B02D1280000F063F9304B9C4201D110
:1093C0006C6808E02E4B9C4201D1AC6803E02D4B49
:1093D0009C4200D1EC68A3899AB2110723D4D1062C
:1093E00007D409220120326037321343A38140425F
:1093F00040E0530713D5616B002908D023004433A4
:10940000994202D03000FFF797FA002363632422C9
:10941000A3899343A3810023636023692360082207
:10942000A3891343A3812369002B0BD1A023A28915
:109430009B00134080229200934203D02100300011
:1094400000F0B2F90123A289134005D00023A360E4
:1094500063695B42A36103E0910700D46369A36081
:1094600000202369834205D1130603D540231A4304
:10947000A281013870BDC04620020020B0AD0000BE
:10948000D0AD0000F0AD000010B5062000F0AEFB3E
:10949000012000F0E3FC0000F7B58A8905000C000C
:1094A00013075AD44B68002B02DC0B6C002B19DD20
:1094B000E76A002F16D000232E682B6080235B0103
:1094C0001A4001D0606D14E00123216A2800B847DA
:1094D000431C0ED12B68002B0BD01D2B01D0162B5B
:1094E00002D12E6000205AE04022A3891343A381B9
:1094F00055E0A3895B0706D56368C01A636B002B30
:1095000001D0236CC01A00230200216A2800E76AF8
:10951000B847A389421C06D129681D293AD8204A98
:10952000CA40D20736D50022626022692260DB047D
:1095300005D5431C02D12B68002B00D16065616BFF
:109540002E600029CED023004433994202D0280057
:10955000FFF7F2F90020606321E00F69002FC1D00E
:109560000B680F60DB1B01930023920700D14B694E
:10957000A36003E0019B3F181B1A0193019B002B82
:10958000B0DD019B3A00216A2800A66AB047002896
:10959000F0DCA389402201201343A3814042FEBD99
:1095A000010040200B6970B505000C00002B01D1B3
:1095B00000201CE0002804D08369002B01D100F0BA
:1095C0005FF80B4B9C4201D16C6808E0094B9C4250
:1095D00001D1AC6803E0084B9C4200D1EC680C223E
:1095E000A35E002BE4D021002800FFF755FF70BDDB
:1095F000B0AD0000D0AD0000F0AD000010B50249E4
:1096000000F0B0F810BDC046A5950000002310B5CD
:10961000040003604360836081814366C28103610B
:1096200043618361190008225C30FFF77CF9054B28
:1096300024626362044BA362044BE362044B236322
:1096400010BDC0462D9C0000559C00008D9C000064
:10965000B99C000070B568254B1E5D430E002900C3
:109660007431FFF7AFF9041E08D000212A00016011
:1096700046600C30A0606832FFF755F9200070BDDD
:10968000836913B50400002B28D18364C364036588
:10969000134B144A1B6882620193984201D1012343
:1096A0008361200000F020F86060200000F01CF8CA
:1096B000A060200000F018F80022E060042160683B
:1096C000FFF7A4FF01220921A068FFF79FFF0222F4
:1096D0001221E068FFF79AFF0123A36113BDC04682
:1096E00078AC0000FD950000F8B51D4B06001D6824
:1096F000AB69002B02D12800FFF7C2FF4835AC68E8
:109700006B68013B05D40C22A75E002F10D0683493
:10971000F7E72B68002B01D02D68F0E7042130001B
:10972000FFF798FF28600028F6D10C23336016E07D
:10973000012320005B42E3810233A3816766276037
:10974000A760676027616761A7615C300822390004
:10975000FFF7E9F820006763A763A764E764F8BD33
:1097600078AC0000F7B504000700002601914834EA
:10977000002C16D06368A5680093009B013B009302
:109780000DD4AB89012B08D90E22AB5E013304D076
:1097900029003800019B984706436835EDE72468A7
:1097A000E6E73000FEBD0000F0B58B8991B0060001
:1097B0000C009B0726D40E23C95E002904DA8023FF
:1097C000A5891D4010D10CE001AA00F0A1FA0028E3
:1097D000F5DBF023029D1B021D401A4BED186B4276
:1097E0005D418027FF0001E000254027390030005F
:1097F000FFF7E8F800280CD1A3899A051FD40222AC
:109800001343A38123004733236023610123636152
:1098100015E080220C4BB362A38920601343A3811F
:1098200020616761002D0AD00E23E15E300000F058
:1098300081FA002803D00122A3891343A38111B028
:10984000F0BDC04600E0FFFFFD950000C9B28218E0
:10985000904204D003788B4202D00130F8E7002018
:10986000704710B5884202D98B18984201D3002363
:1098700005E09B1A013A08D3995C8154FAE79342B8
:1098800003D0CC5CC4540133F9E710BDF8B5060031
:109890000C001500002904D11100FFF793F8040013
:1098A00018E0002A03D1FFF747F82C0012E000F07F
:1098B00067FA85420ED929003000FFF783F8071EAA
:1098C00007D021002A00FFF725F821003000FFF71C
:1098D00033F83C002000F8BDF0B58E6885B0070075
:1098E0000C00039201939E4243D890238A89DB00A7
:1098F0001A423ED003250969236801985B1A029336
:1099000063695D43EB0F5D19029B6D1001331B18FA
:10991000AB4200D91D00530510D529003800FFF7D0
:1099200051F8061E14D0029A2169FEF7F3FFA289AE
:10993000194B134080221343A38112E02A00380000
:10994000FFF7A4FF061E0CD121693800FEF7F4FFD3
:109950000C23402201203B60A38940421343A38192
:1099600017E0029B2661F61826606561019EED1ADC
:10997000A560019BB34200D21E003200039920680B
:10998000FFF76FFF0020A3689B1BA36023689E194D
:10999000266005B0F0BDC0467FFBFFFFF0B59FB06D
:1099A000029005938B890F0016001B0610D50B69DA
:1099B000002B0DD14021FFF705F8386038610028F1
:1099C00004D10C23029A01381360D8E040237B6154
:1099D000002306AD6B6120336B761033AB76340019
:1099E0002378002B03D1A31B049312D003E0252B73
:1099F000F9D00134F4E7A31B320039000298FFF7D5
:109A00006BFF431C00D1B4E06A69049B9446634435
:109A10006B612378002B00D1ABE00122002352427E
:109A20006A6002A95432521801342B60EB60AB60BB
:109A30001370AB65534E217805223000FFF706FF07
:109A4000002807D00123801B83402A680134134378
:109A50002B60EFE72B68DA0604D55322202102A8F9
:109A6000121811701A0704D553222B2102A81218BC
:109A7000117022782A2A03D0099B00200A210EE0C7
:109A8000059A111D12680591002A01DB099204E074
:109A90005242EA60022213432B6001340BE0227829
:109AA000303A092A04D84B4301349B180120F6E7C9
:109AB000002800D0099323782E2B1ED163782A2BFF
:109AC0000AD1059B02341A1D1B680592002B01DA8E
:109AD00001235B42079310E000230A201A0001349F
:109AE0006B6021783039092904D842430134521877
:109AF0000123F6E7002B00D00792234E21780322A2
:109B00003000FFF7A3FE002806D04023801B8340CF
:109B10002A68013413432B60217806221B48661CF7
:109B20002976FFF793FE002812D0194B002B06D19F
:109B30000722059B073393430833059314E005ABD5
:109B400000933A00134B2900029800E000BF07E0A1
:109B500005AB00933A000F4B29000298FFF73AF942
:109B60000390039B013304D06B69039A9B186B61CC
:109B700035E7BB890B985B0601D5012040421FB039
:109B8000F0BDC0467CAC000082AC000086AC00009A
:109B900000000000D998000070B504000D1E1F2DB4
:109BA00004D916230360012040421EE0426C002AC3
:109BB00004D08B00D2181368002B08D1200000F0CD
:109BC00031F82A000100200000F01AF80DE0002012
:109BD000012B0AD0591C03D117332360013004E054
:109BE0000024280014609847200070BD10B5034B76
:109BF00001001868FFF7D0FF10BDC046200200200A
:109C0000002370B5064C050008001100236000F029
:109C1000F7F8431C03D12368002B00D02B6070BDE4
:109C2000EC24002010B500F0DBF810BD70B50C007E
:109C30000E25495F00F0B0F8002803DB636D1B18A8
:109C4000636503E0A289024B1340A38170BDC04647
:109C5000FFEFFFFFF8B51F008B8905000C00160011
:109C6000DB0505D50E23C95E0022022300F074F83F
:109C7000A289054B28001340A38132000E23E15E28
:109C80003B0000F01FF8F8BDFFEFFFFF70B50C00C0
:109C90000E25495F00F060F8A389421C03D1054AF4
:109CA0001340A38104E0802252011343A381606525
:109CB00070BDC046FFEFFFFF10B50E23C95E00F078
:109CC00015F810BD70B50500080011000022064C03
:109CD00022601A0000F0BAF8431C03D12368002B5D
:109CE00000D02B6070BDC046EC240020002370B56E
:109CF000064C05000800236000F062F8431C03D105
:109D00002368002B00D02B6070BDC046EC240020DF
:109D1000002370B5064C050008001100236000F018
:109D200057F8431C03D12368002B00D02B6070BD73
:109D3000EC240020002370B5064C050008002360C9
:109D400000F056F8431C03D12368002B00D02B6091
:109D500070BDC046EC24002070B50500080011005D
:109D60000022064C22601A0000F052F8431C03D176
:109D70002368002B00D02B6070BDC046EC2400206F
:109D80000B1F1A68101F002A04DA891804390B689F
:109D9000D01804387047000070B5050008001100A5
:109DA0000022064C22601A0000F03AF8431C03D14E
:109DB0002368002B00D02B6070BDC046EC2400202F
:109DC00058220120014B40421A607047EC240020C9
:109DD00058220120014B40421A607047EC240020B9
:109DE00058220120014B40421A607047EC240020A9
:109DF0005822024B00201A607047C046EC24002015
:109E000058220120014B40421A607047EC24002088
:109E100058220120014B40421A607047EC24002078
:109E200058220120014B40421A607047EC24002068
:109E3000044A1368002B03D01818106018007047EC
:109E4000014BF9E7FC110020F024002058220120EA
:109E5000014B40421A607047EC240020FEE7C046E8
:109E6000F8B5C046F8BC08BC9E467047F8B5C04679
:109E7000F8BC08BC9E4670478E0600002006000015
:109E80009E060000D4060000100700004A070000EC
:109E900086070000AE070000EC0700003208000053
:109EA0008E080000D2080000380900008409000074
:109EB000AC090000E6090000300A0000580A000062
:109EC000900A0000CA0A0000060B00008C0B00007C
:109ED000540C0000E40C0000420D0000840D000052
:109EE000A60D0000AE0D0000900E00008E060000D2
:109EF0008E0600008E0600008E060000DC0E0000BC
:109F0000460F0000B00F0000FA0F00005C100000C8
:109F1000E210000070110000BE11000008120000E5
:109F2000401200008C120000D81200002413000020
:109F300072130000C813000008140000741400001D
:109F4000A6140000F21400003E1500008A1500005F
:109F5000C6150000121600005E1600008E060000F6
:109F60008E0600008E060000C8160000FA160000DB
:109F70002C1700005817000094170000C0170000AD
:109F80008E0600008E0600008E0600008E06000081
:109F9000F21700003A1800008E0600008E0600003E
:109FA00086180000B4180000FE1800008E0600009D
:109FB0008E0600008E0600002E19000060190000B9
:109FC00092190000C4190000F0190000281A0000BE
:109FD000541A00007E1A0000A81A0000DA1A0000C5
:109FE0000C1B00004C1B0000781B0000AA1B00008B
:109FF000D61B00008E0600008E0600008E060000B4
:10A000008E0600008E060000081C0000341C0000B4
:10A01000601C00008C1C0000B81C0000F01C00003C
:10A02000281D0000601D0000981D0000C41D0000D8
:10A03000F21D0000241E00008E0600008E060000A7
:10A040008E0600008E0600008E0600008E060000C0
:10A050008E0600008E0600008E0600008E060000B0
:10A060008E0600008E0600008E0600008E060000A0
:10A07000521E0000801E000066616C7365007472E1
:10A080007565006C697374206F662025642069749F
:10A09000656D73006F626A656374206F6620636C20
:10A0A0006173733A20256400537461636B20756E8D
:10A0B000646572666C6F77000D0A564D2050616EB4
:10A0C00069633A2025730D0A00496E7375666669E7
:10A0D0006369656E74206D656D6F727920666F724D
:10A0E000204D6963726F426C6F636B73206F626A9D
:10A0F000656374206865617000496E737566666992
:10A100006369656E74206D656D6F727920666F721C
:10A11000204D6963726F426C6F636B73207374615F
:10A12000636B00626164206F626A656374206174AE
:10A1300020256C640A0025783A20256420776F7208
:10A1400064732C20636C61737349442025640A0096
:10A150004865616465723A2025780A0009307825DF
:10A16000782C0A006D6973630073696E00256420A2
:10A1700025642025642025640A00426164207265FC
:10A18000636F726420666F756E6420647572696EA9
:10A190006720696E697469616C697A6174696F6E50
:10A1A000210A004E6F7420656E6F75676820726FAC
:10A1B0006F6D206576656E20616674657220636FD1
:10A1C0006D70616374696F6E0A00526573746F72AB
:10A1D000696E6720256420736372697074732E2E14
:10A1E0002E0053746172746564002D2D2D2D2D0A7F
:10A1F0000050657273697374656E74204D656D6F80
:10A20000727920546573740A0A000A496E69746988
:10A21000616C697A696E67204D656D6F72790A00AD
:10A220004D656D6F727920696E74697469616C69CE
:10A230007A65643B2077726974696E672072656322
:10A240006F7264732E2E2E0A005265636F72642043
:10A250006174206F66667365742025643A202564F6
:10A260002025642025642025642028256420776F1C
:10A27000726473290A0046696E616C3A20637572D4
:10A2800072656E74202564207573656420256420D2
:10A2900063302025642063312025640A00E2ECF05D
:10A2A000F4F8FC00046E756D626572006E6F6E6589
:10A2B000006F74686572007061697200737472690E
:10A2C0006E6700726164696F0064697361626C65D6
:10A2D000526164696F006D65737361676552656390
:10A2E0006569766564007061636B6574526563656A
:10A2F000697665007061636B657453656E640072A6
:10A3000065636569766564496E7465676572007238
:10A31000656365697665644D6573736167655479D6
:10A320007065007265636569766564537472696E01
:10A33000670073656E64496E746567657200736566
:10A340006E64506169720073656E64537472696EF5
:10A3500067007365744368616E6E656C0073657445
:10A3600047726F757000736574506F776572007314
:10A3700069676E616C537472656E677468004E6FC6
:10A380002066726565207461736B20656E747269F6
:10A3900065730057656C636F6D6520746F204D6940
:10A3A00063726F426C6F636B7321004D656D6F72EA
:10A3B0007920636C65617265642E00416C6C207459
:10A3C00061736B732073746F7070656400763035E1
:10A3D00037002025732025730000000007000000CF
:10A3E000030000006D6963726F3A6269740068610E
:10A3F00073546F6E6500706C6179546F6E650068A0
:10A400006173536572766F00736574536572766F0E
:10A410000000000000000000010000000200000039
:10A4200003000000040000000A0000006E657400D4
:10A43000686173576946690073746172745769463D
:10A44000690073746F70576946690077696669536C
:10A450007461747573006D794950416464726573F9
:10A4600073007468696E67446573637269707469B8
:10A470006F6E00636C6561725468696E67446573E2
:10A480006372697074696F6E00617070656E645498
:10A490006F5468696E674465736372697074696F3D
:10A4A0006E00617070656E64546F5468696E6750B9
:10A4B000726F7065727479001A1B1C030406070919
:10A4C0000A1718191A1B1C03040607090A1718197A
:10A4D000646973706C6179006C696768744C657647
:10A4E000656C000000000000010000000200000098
:10A4F000030000000400000005000000060000004A
:10A500000700000008000000090000000A00000029
:10A510000B0000000C0000000D0000000E00000009
:10A520000F000000100000001200000014000000E6
:10A5300016000000180000001A0000001C000000B7
:10A540001E00000020000000230000002600000084
:10A55000290000002C0000002F0000003200000045
:10A56000360000003A0000003E00000042000000FB
:10A57000460000004B0000005000000055000000A5
:10A580005A00000061000000680000006F00000039
:10A59000760000007D000000840000008B000000B9
:10A5A0009200000099000000A0000000A700000039
:10A5B000AE000000B5000000BC000000C3000000B9
:10A5C000CA000000D1000000D8000000DF00000039
:10A5D000E6000000ED000000F4000000FB000000B9
:10A5E000FF000000000000000008080800080A4AF8
:10A5F0004000000A5FEA5FEA0ED92ED36E1932449A
:10A6000089330C924C924D08080000000488080819
:10A61000040804848488000A448A4000048EC480AC
:10A62000000000048800000EC000000000080001C7
:10A63000224488100C9252524C048C84848E1C82CA
:10A640004C901E1EC244924C06CA525FE21FF01E7E
:10A65000C13E02448ED12E1FE24488100ED12ED16D
:10A660002E0ED12EC4880008000800000480048843
:10A670000244880482000EC00EC008048244880E82
:10A68000D126C0040ED135B36C0C925ED2521C920E
:10A690005C925C0ED010100E1C9252525C1ED01CAC
:10A6A000901E1ED01C90100ED013712E12525ED22E
:10A6B000521C8808081C1FE242524C1254981492F3
:10A6C000101010101E113B75B131113935B3710CDA
:10A6D0009252524C1C925C90100C92524C861C92DE
:10A6E0005C92510ED00C825C1FE48484841252521E
:10A6F000524C1131312A44113135BB7112524C92F6
:10A7000052112A4484841EC488101E0EC808080EE4
:10A7100010080482410EC242424E048A40000000EA
:10A720000000001F0804800000000ED2524F1010DD
:10A730001C925C000ED0100E02424ED24E0C925C67
:10A74000900E06C81C88080ED24EC24C10101C92E7
:10A75000520800080808024002424C101498149253
:10A760000808080806001B75B131001C92525200FF
:10A770000C92524C001C925C90000ED24EC2000E05
:10A78000D010100006C8049808080EC8070012521E
:10A79000524F0011312A4400113135BB00124C8C4C
:10A7A0009200112A4498001EC4881E06C48C848618
:10A7B000080808080818080C881800000C83607343
:10A7C000656E736F72730074656D70657261747518
:10A7D00072650074696C74580074696C7459007403
:10A7E000696C745A00746F756368526561640069BE
:10A7F000326352656164006932635772697465003F
:10A8000074667400656E61626C65446973706C6136
:10A810007900736574506978656C006C696E6500C9
:10A820007265637400726F756E64656452656374FB
:10A8300000636972636C6500747269616E676C6550
:10A84000007465787400535049436C6173733A3AED
:10A85000535049436C617373284E52465F535049BD
:10A860005F547970652A2C2075696E74385F742C7A
:10A870002075696E74385F742C2075696E74385F4A
:10A88000742900705F73706920213D204E554C4C37
:10A89000002F55736572732F6A6F686E6D616C6FF0
:10A8A0006E65792F4C6962726172792F417264759D
:10A8B000696E6F31352F7061636B616765732F73DC
:10A8C000616E646565706D69737472792F68617209
:10A8D00064776172652F6E5246352F302E362E30DA
:10A8E0002F6C69627261726965732F5350492F53DF
:10A8F00050492E637070000000000000000000004E
:10A900004B4B0000114B0000374B0000414B000047
:10A91000714B0000354B00000300000002000000F6
:10A92000010000000400000005000000110000000C
:10A930000C0000000B000000120000000A000000E4
:10A94000060000001A0000001400000017000000BC
:10A95000160000001500000010000000FFFFFFFFC0
:10A96000FFFFFFFF000000001E00000019000000B4
:10A9700018000000070000000800000009000000A7
:10A980000D0000000E0000000F0000001C00000081
:10A990001B0000001D00000013000000000000006C
:10A9A000000000000000304300000000000030C341
:10A9B000FB21F93FFB2109407CD91240FB211940C2
:10A9C0007A6A1F407CD92240BBFD2540FB212940EB
:10A9D0003A462C407A6A2F405C4731407CD932405D
:10A9E0009C6B3440BBFD3540DB8F3740FB21394049
:10A9F0001BB43A403A463C405AD83D407A6A3F4000
:10AA00004C7E40405C4741406C1042407CD9424003
:10AA10008CA243409C6B4440AC344540BBFD454058
:10AA2000CBC64640DB8F4740EB584840FB214940AE
:10AA300083F9A200444E6E00FC291500D15727006F
:10AA4000DD34F50062DBC0003C9995004190430085
:10AA50006351FE00BBDEAB00B761C5003A6E240057
:10AA6000D24D42004906E00009EA2E001C92D100B6
:10AA7000EB1DFE0029B11C00E83EA700F535820061
:10AA800044BB2E009CE98400B4267000417E5F0028
:10AA9000D6913900538339009CF439008B5F8400D0
:10AAA00028F9BD00F81F3B00DEFF97000F98050056
:10AAB000112FEF000A5A8B006D1F6D00CF7E3600FC
:10AAC00009CB2700464FB7009E663F002DEA5F0086
:10AAD000BA277500E5EBC7003D7BF100F7390700A9
:10AAE00092528A00FB6BEA001FB15F00085D8D0087
:10AAF000300356007BFC4600F0AB6B0020BCCF005F
:10AB000036F49A00E3A91D005E619100081BE6007F
:10AB100085996500A0145F008D40680080D8FF0013
:10AB200027734D0006063100CA561500C9A87300E8
:10AB30007BE260006B8CC00002000000030000009C
:10AB4000040000000600000000000040FB21F93F67
:10AB5000000000002D44743E000000809846F83C40
:10AB60000000006051CC783B00000080831BF0396E
:10AB70000000004020257A38000000802282E33661
:10AB8000000000001DF36935000000000000000017
:10AB90008D670000AD660000FD67000011680000D1
:10ABA000076800008B6700007F6700001D680000D9
:10ABB000A96700007B67000094700000F26F00003E
:10ABC000F26F0000F06F00008670000086700000D9
:10ABD0007C700000F06F0000867000007C70000048
:10ABE00086700000F06F00008C7000008C70000018
:10ABF0008C70000016710000947C0000547B0000F3
:10AC0000547B0000527B00006C7C00006C7C0000D8
:10AC10005E7C0000527B00006C7C00005E7C0000CB
:10AC20006C7C0000527B0000747C0000747C00008F
:10AC3000747C0000747E00002C2066756E6374695D
:10AC40006F6E3A2000617373657274696F6E2022B3
:10AC5000257322206661696C65643A2066696C65BB
:10AC600020222573222C206C696E652025642573B3
:10AC700025730A0043000000C0010020232D302B63
:10AC80002000686C4C0065666745464700303132ED
:10AC90003334353637383941424344454600303144
:10ACA00032333435363738396162636465660000A3
:10ACB000202020202020202020282828282820206C
:10ACC0002020202020202020202020202020202084
:10ACD00088101010101010101010101010101010FC
:10ACE00004040404040404040404101010101010DC
:10ACF00010414141414141010101010101010101B5
:10AD000001010101010101010101011010101010E8
:10AD10001042424242424202020202020202020285
:10AD200002020202020202020202021010101020AD
:10AD30000000000000000000000000000000000013
:10AD40000000000000000000000000000000000003
:10AD500000000000000000000000000000000000F3
:10AD600000000000000000000000000000000000E3
:10AD700000000000000000000000000000000000D3
:10AD800000000000000000000000000000000000C3
:10AD900000000000000000000000000000000000B3
:10ADA00000000000000000000000000000000000A3
:10ADB0000000000000000000000000000000000093
:10ADC0000000000000000000000000000000000083
:10ADD0000000000000000000000000000000000073
:10ADE0000000000000000000000000000000000063
:10ADF0000000000000000000000000000000000053
:10AE00000000000000000000000000000000000042
:04AE1000000000003E
:08AE14006053FF7F0100000004
:10AE1C00FFFFFFFF69A10000B9200000C9A20000DC
:10AE2C008D270000D6A20000A52A0000E6A2000093
:10AE3C00452A0000F4A20000312C0000FFA2000003
:10AE4C00A92700000FA300001128000023A3000075
:10AE5C00B927000032A300004B2D00003EA30000D8
:10AE6C00D52C000047A300007B2C000052A300004F
:10AE7C00C12900005DA300004929000066A3000061
:10AE8C007D2900006FA30000C127000019FCFFFF03
:10AE9C00FFFFFFFFEEA30000CD390000F6A300007A
:10AEAC00C9390000FFA30000D139000008A400003C
:10AEBC00D539000030A40000953C000038A40000F7
:10AECC00C53C000042A40000D93C00004BA400008B
:10AEDC00E33C000056A40000CF3C000062A400003C
:10AEEC00A33C000073A40000B93C000089A400003E
:10AEFC00AD3C0000A2A40000993C0000D8A40000C6
:10AF0C00053D000018000000FF000000C7A700006E
:10AF1C0015450000D3A7000081480000D9A7000008
:10AF2C0091480000DFA70000A1480000E5A7000041
:10AF3C0049450000EFA70000B1480000F7A700004A
:10AF4C008946000004A800003D49000012A800003A
:10AF5C00414900001BA800004549000020A8000042
:10AF6C004949000025A800004D49000031A8000007
:10AF7C005149000038A800003949000041A80000E0
:10AF8C00354900000300000002000000080000002A
:10AF9C000A000000FFFFFFFF00000000010000009E
:10AFAC000000020001000000FFFFFFFF0000000096
:10AFBC00020000000000040002000000FFFFFFFF81
:10AFCC000000000003000000000008000300000067
:10AFDC0000000000B0AD0000D0AD0000F0AD0000EE
:10AFEC000000000000000000000000000000000055
:10AFFC0074AC000000000000000000000000000025
:10B00C000000000000000000000000000000000034
:10B01C000000000000000000000000000000000024
:10B02C000000000000000000000000000000000014
:10B03C00C0010020AFAC000039010000E14A000063
:10B04C00014E0000816A00000D01000000000000AC
:040000030000623D5A
:00000001FF
